:100000000C94B7010C9447310C9474310C94DF01BB
:100010000C94DF010C94DF010C94DF010C94DF01E0
:100020000C94DF010C94DF010C94DF010C94CA06E0
:100030000C94DF010C94DF010C94DF010C94DF01C0
:100040000C9453300C94DF010C9440060C947C0605
:100050000C94DF010C94DF010C94DF010C94DF01A0
:100060000C94DF010C94DF01084AD73B3BCE016EB4
:1000700084BCBFFDC12F3D6C74319ABD56833DDAFF
:100080003D00C77F11BED9E4BB4C3E916BAAAABE0E
:10009000000000803F05A84CCDB2D44EB93836A937
:1000A000020C50B9918688083CA6AAAA2ABE000074
:1000B00000803F0664EC1B3C04BC163E3BE5B93CAB
:1000C000C93C37C29E5A3D660498083EEA69AAAA0E
:1000D0003E000000803F2020BF0020BF00BF007C0A
:1000E0002020202020202020202020202020202010
:1000F00020202000C8202020202020202020202078
:1001000020C900C8202020202020202020202020BE
:10011000C97C00D820202020202020202020202042
:10012000D97C00C820202020202020202020202032
:10013000C97C00C820202020202020202020202032
:10014000C97C00207265766F006D696E6F706F7389
:1001500064206C6962726570696C6F740020202085
:100160002020BABBBCBDBE7C2020202020CACBCC26
:10017000CDCE7C00626F6F74696E672075703AED4A
:10018000F2F2F2F2F2F2F2F30062617474657279E3
:10019000207761726E696E672000747870696420E0
:1001A00076616C756573006261726F2074656D7045
:1001B0000074656D706469737020006163746976A2
:1001C000652000706173736976650075617674618E
:1001D0006C6B200073657475702073637265656E57
:1001E0007C7C7C004368617220446F6E650A00521B
:1001F0006561647920666F7220466F6E740A0055DF
:1002000070646174652043686172536574000040D6
:100210007A10F35A00A0724E18090010A5D4E80015
:1002200000E87648170000E40B54020000CA9A3B2D
:10023000000000E1F50500008096980000004042B3
:100240000F000000A0860100000010270000000041
:10025000E803000000006400000000000A00000045
:1002600000000100000000002C76D888DC674F08F1
:1002700023DFC1DFAE59E1B1B796E5E3E453C63AF7
:10028000E651997696E8E6C28426EB898C9B62ED6E
:10029000407C6FFCEFBC9C9F40F2BAA56FA5F49028
:1002A000055A2AF75C936B6CF9676DC11BFCE0E49F
:1002B0000D47FEF520E6B500D0ED902E03009435F5
:1002C00077050080841E080000204E0A000000C848
:1002D0000C333333330F986E12831141EF8D211499
:1002E000893BE65516CFFEE6DB18D1844B381BF769
:1002F0007C1D901DA4BBE424203284725E22810008
:10030000C9F124ECA1E53D276E616E00696E6600BF
:1003100000000000240027002A0000000000250043
:1003200028002B0000000000230026002900040400
:10033000040404040404020202020202030303038D
:100340000303010204081020408001020408102069
:100350000102040810200000000700020100000351
:10036000040600000000000000004B0411081124E6
:100370001FBECFEFD8E0DEBFCDBF13E0A0E0B1E0FD
:10038000E6E3FDE602C005900D92A83DB107D9F75E
:1003900016E0A8EDB3E001C01D92A938B107E1F75E
:1003A00013E0CEE6D3E004C02297FE010E9495360A
:1003B000CA36D107C9F70E945E320C9499360C9464
:1003C0000000FA01AA27283051F1203181F1E89488
:1003D0006F936E7F6E5F7F4F8F4F9F4FAF4FB1E038
:1003E0003ED0B4E03CD0670F781F891F9A1FA11D33
:1003F000680F791F8A1F911DA11D6A0F711D811D34
:10040000911DA11D20D009F468943F912AE0269FF8
:1004100011243019305D3193DEF6CF010895462F57
:100420004770405D4193B3E00FD0C9F7F6CF462F38
:100430004F70405D4A3318F0495D31FD40524193A1
:1004400002D0A9F7EACFB4E0A6959795879577955E
:100450006795BA95C9F700976105710508959B01E5
:10046000AC010A2E06945795479537952795BA956E
:10047000C9F7620F731F841F951FA01D08952830B0
:1004800008F027E03327DA01990F311D87FD9160CD
:1004900000966105710539F432602E5F3D9330E3BB
:1004A0002A95E1F708959F3F30F080387105610586
:1004B00009F03C5F3C5F3D93913008F08068911DEE
:1004C000DF93CF931F930F93FF92EF92192F987F93
:1004D0009695E92F96959695E90FFF27E859FD4FD8
:1004E00099273327EE24FF24A701E70105900894FC
:1004F000079428F4360FE71EF81E491F511D660F9A
:10050000771F881F991F0694A1F70590079428F478
:10051000E70EF81E491F561FC11D770F881F991F30
:10052000661F0694A1F70590079428F4F80E491F5A
:10053000561FC71FD11D880F991F661F771F06946E
:10054000A1F70590079420F4490F561FC71FD81F25
:10055000990F661F771F881F0694A9F7849110953D
:10056000177041F0D695C79557954795F794E7943E
:100570001A95C1F7EEE0F2E0689415901591359167
:100580006591959105907FE27395E118F10A430B0F
:10059000560BC90BD009C0F7E10CF11E431F561FC3
:1005A000C91FD01D7EF4703311F48A95E6CFE8940C
:1005B000015030F0080F0AF40027021708F4202F2A
:1005C0002395022F7A3328F079E37D932A95E9F772
:1005D00010C07D932A9589F606949795679537956F
:1005E00017951794E118F10A430B560BC90BD00964
:1005F00098F023957E9173957A3308F070E37C939D
:100600002013B8F77E9170617D9330F0839571E38C
:100610007D9370E32A95E1F71124EF90FF900F91FD
:100620001F91CF91DF91992787FD90950895CF93E2
:10063000DF93BC018230910510F462E070E0A0917C
:100640008706B0918806ED0140E050E0E0E0F0E080
:1006500021C0888199818617970769F48A819B81D7
:10066000309719F09383828304C090938806809317
:100670008706FE0134C06817790738F44115510523
:1006800019F08417950708F4AC01FE018A819B815B
:100690009C01E9012097E9F641155105A9F1CA012C
:1006A000861B970B049708F4BA01E0E0F0E02AC03B
:1006B0008D919C91119784179507F9F4641775072C
:1006C00081F412968D919C911397309719F0938332
:1006D000828304C09093880680938706FD0132963A
:1006E0004CC0CA01861B970BFD01E80FF91F6193EF
:1006F000719302978D939C9340C0FD0182819381F9
:100700009C01D9011097A1F68091850690918606EB
:10071000892B41F48091790290917A029093860618
:100720008093850640917B0250917C0241155105D2
:1007300041F44DB75EB78091770290917802481BE3
:10074000590B2091850630918606CA01821B930BB6
:100750008617970780F0AB014E5F5F4F84179507B0
:1007600050F0420F531F5093860640938506F901BF
:100770006193719302C0E0E0F0E0CF01DF91CF918F
:100780000895CF93DF93009709F450C0EC012297AE
:100790001B821A82A0918706B0918806109709F1F2
:1007A00040E050E0AC17BD0708F1BB83AA83FE010F
:1007B00021913191E20FF31FAE17BF0779F48D91AC
:1007C0009C911197280F391F2E5F3F4F3983288343
:1007D00012968D919C9113979B838A8341155105A5
:1007E00071F4D0938806C093870620C012968D912D
:1007F0009C911397AD01009711F0DC01D3CFFA0162
:10080000D383C28321913191E20FF31FCE17DF070B
:1008100069F488819981280F391F2E5F3F4FFA01B3
:10082000318320838A819B8193838283DF91CF915F
:100830000895FC010590615070400110D8F7809533
:1008400090958E0F9F1F0895FC016150704001909C
:100850000110D8F7809590958E0F9F1F08956EBD5B
:100860000DB407FEFDCF8EB508958DE061E00E94C6
:10087000A1318BE061E00E94A1318CE060E00E9438
:10088000A1318AE061E00E94A1311CBC80E58CBDF1
:100890008DB58EB5089588ED93E00E9435040895D6
:1008A000FC011382128288EE93E0A0E0B0E0848322
:1008B0009583A683B7838DE892E091838083089522
:1008C000FC018089803419F421E030E002C020E08E
:1008D00030E0C9010895FC01818990E00895FC0190
:1008E0006487458766874787089580E090E008958C
:1008F00080E090E0089580E090E008950895EF9200
:10090000FF921F93CF93DF93162F7A0186E060E06A
:100910000E94E03188ED93E060E00E942F0488EDB2
:1009200093E060E00E942F0488ED93E069E00E946C
:100930002F0488ED93E0612F0E942F04C0E0D0E0E7
:10094000F701EC0FFD1F108188ED93E06AE00E9433
:100950002F0488ED93E06C2F0E942F0488ED93E024
:100960006BE00E942F0488ED93E0612F0E942F041A
:100970002196C633D10521F788ED93E068E00E9407
:100980002F0488ED93E060EA0E942F0488ED93E045
:1009900060EA0E942F0485FDF9CF88ED93E060E0C6
:1009A0000E942F0488ED93E06CE00E942F0486E003
:1009B00061E00E94E031DF91CF911F91FF90EF90B5
:1009C00008951F93CF93DF93EC01162F86E060E02C
:1009D0000E94E03188ED93E060E00E942F04112333
:1009E00019F0113059F404C088ED93E0688904C00F
:1009F00068896C6188ED93E00E942F0486E061E0D5
:100A00000E94E031DF91CF911F910895EF92FF9204
:100A10000F931F938EE1489F70011124E60EF11C85
:100A200086E060E00E94E03108ED13E0C80165E077
:100A30000E942F04C8016F2D0E942F04C80166E098
:100A40000E942F04C8016E2D0E942F041F910F9148
:100A5000FF90EF900895EF92FF920F931F937C0108
:100A600008ED13E0C80167E00E942F04C8016FEF92
:100A70000E942F0486E061E00E94E031F701878543
:100A80008F5F87871F910F91FF90EF900895EF92EE
:100A9000FF920F931F93FC01E7848EE1E89E7001A3
:100AA00011248685E80EF11C86E060E00E94E031AA
:100AB00008ED13E0C80164E00E942F04C80163E060
:100AC0000E942F04C80165E00E942F04C8016F2D09
:100AD0000E942F04C80166E00E942F04C8016E2DF9
:100AE0000E942F041F910F91FF90EF9008951F9384
:100AF000CF93DF93EC01162F6C3731F40E942B0556
:100B0000CE010E9447050AC088ED93E067E00E948D
:100B10002F0488ED93E0612F0E942F0481E090E084
:100B2000DF91CF911F9108950F931F9386E060E0AE
:100B30000E94E03108ED13E0C80164E00E942F0438
:100B4000C80164E00E942F0486E061E00E94E03169
:100B50001F910F9108951F93CF93DF93EC01188A93
:100B600016E0198B85E796E060E973E00E94B32FE9
:100B7000813049F480E4888B88E0898B86E060E0EE
:100B80000E94E03102C0188A198B86E060E00E9462
:100B9000E031DF91CF911F9108950F931F93CF9371
:100BA000DF93EC0186E061E00E94A13182E060E029
:100BB0000E94A13182E061E00E94E031CE010E94FA
:100BC000AB0586E060E00E94E03188ED93E06CEEDA
:100BD0000E942F0488ED93E06FEF0E942F04182FDE
:100BE00088ED93E060E00E942F046889626088EDE0
:100BF00093E00E942F0462E370E080E090E00E94A6
:100C0000A93088ED93E06CE60E942F041F7E88EDEA
:100C100093E0612F0E942F048889803419F00DE041
:100C200010E002C000E110E01092DA031092D90344
:100C300017C06091D9037091DA03605F88ED93E08B
:100C40000E942F0488ED93E069E00E942F048091B8
:100C5000D9039091DA0301969093DA038093D90334
:100C60008091D9039091DA038017910714F3CE0194
:100C700061E00E94E104DF91CF911F910F910895EF
:100C80001F920F920FB60F9211242F933F934F9301
:100C90008F939F93EF93FF934091C600209164063A
:100CA000309165062F5F3F4F8091680690916906ED
:100CB0002823392380916606909167062817390703
:100CC00079F08091640690916506E0916A06F09152
:100CD0006B06E80FF91F4083309365062093640686
:100CE000FF91EF919F918F914F913F912F910F9095
:100CF0000FBE0F901F9018951F920F920FB60F9274
:100D000011242F933F938F939F93EF93FF93209101
:100D10006E0630916F0680916C0690916D062817D3
:100D20003907E9F080916E0690916F06E0917206A6
:100D3000F0917306E80FF91F80818093C6008091BF
:100D40006E0690916F0601962091700630917106A3
:100D50008223932390936F0680936E0610C0209198
:100D60006C0630916D0680916E0690916F06281783
:100D7000390729F48091C1008F7D8093C100FF91D4
:100D8000EF919F918F913F912F910F900FBE0F90F8
:100D90001F9018951F920F920FB60F9211248F93E8
:100DA0009F9380919B0490919C04892B51F080919A
:100DB0009D0490919E04019690939E0480939D04BF
:100DC00009C080919F049091A00401969093A00483
:100DD00080939F049F918F910F900FBE0F901F9053
:100DE0001895CF93DF93482FEB018091FB0583305B
:100DF00009F45DC0843028F48130C1F0823058F5A8
:100E00000AC0853009F4D2C0853008F4A8C0863005
:100E100009F0F2C0E9C04C3309F0EEC081E08093E4
:100E2000FB05488384EB8093FA05E6C0842F90E0AD
:100E3000E091FA05F0E0E827F927E556FD4F20811B
:100E40002093FA05887F9070809741F582E0809327
:100E5000FB05498329C0242F30E0E091FA05F0E03A
:100E6000E227F327E556FD4F80818093FA058091B4
:100E7000F9058F5F8093F905823018F43B832A834C
:100E8000BBC0922F88272A813B81820F931F9B83AF
:100E90008A830A978F3F910521F018F01092FB0585
:100EA000ABC083E08093FB051092F905A5C0E42F49
:100EB000F0E08091FA0590E0E827F927E556FD4F2C
:100EC00080818093FA056091F9056F5F6093F90561
:100ED000623089F0633020F4613009F08DC006C0C3
:100EE000633091F0643009F087C022C0842F90E015
:100EF000A0E0B0E018C0242F30E040E050E0542FD4
:100F0000432F322F222707C0242F30E040E050E04B
:100F1000A901332722278C819D81AE81BF81820F59
:100F2000931FA41FB51F8C839D83AE83BF8364C0B2
:100F3000242F30E040E050E0522F4427332722276F
:100F40008C819D81AE81BF81820F931FA41FB51F2D
:100F50008C839D83AE83BF836093FB05A5CF242F35
:100F600030E0E091FA05F0E0E227F327E556FD4F87
:100F700080818093FA058091F9058F5F8093F90550
:100F8000813019F08230C1F503C03987288734C019
:100F9000922F882728853985280F391F3987288778
:100FA0008A819B810A97F1F085E07CCFE42FF0E005
:100FB0008091FA0590E0E827F927E556FD4F8081FA
:100FC0008093FA052091F9052F5F2093F90530E011
:100FD000FB01E20FF31F41878A819B810A97281743
:100FE000390750F086E05ECFC75FDE4F4883C950B7
:100FF000D14087E08093FB058091FB05873069F441
:101000001092FB05C75FDE4F9091FA058881C950A9
:10101000D140981711F48A8101C080E0DF91CF910F
:1010200008958F92AF92CF92EF92FF920F931F93FA
:1010300081E694E060E045EC50E024EC30E000EC28
:1010400010E0B1ECEB2EF12CCC24C394A8E9AA2E2D
:10105000F0E28F2E0E9423298EE794E00E94500434
:10106000109291041092920410929304109294049E
:10107000109295041092960410929704109298047E
:1010800010929A0410929904109290041F910F915B
:10109000FF90EF90CF90AF908F900895AF92BF9256
:1010A000CF92DF92EF92FF920F931F93E090600632
:1010B000F090610600916206109163068FE590E062
:1010C000A0E0B0E0E80EF91E0A1F1B1F0E949B3033
:1010D0006E157F058007910708F44EC0A090C604E6
:1010E000B090C704C090C804D090C904C601B5012F
:1010F00020E030E040E85FE30E94FE34181694F5EB
:10110000E0901806F090190600911A0610911B063F
:101110000E949B30209160063091610640916206EA
:1011200050916306621B730B840B950B0E94D433A2
:101130009B01AC01C601B5010E94093520E030E0F9
:101140004AE754E40E943B339B01AC01C801B7015C
:101150000E946E32609318067093190680931A06E7
:1011600090931B060E949B3060936006709361060B
:1011700080936206909363061F910F91FF90EF900A
:10118000DF90CF90BF90AF900895DF93CF9300D0C2
:1011900000D0CDB7DEB7FB01E80FF91F628583856C
:1011A0009485258569838A839B832C83492F5C8161
:1011B000782FCA010F900F900F900F90CF91DF9171
:1011C0000895AF92BF92DF92EF92FF920F931F9319
:1011D000CF93DF938C018091FC0580FDE4C0F80182
:1011E000F08081E694E06F2D0E94042AE801C75F39
:1011F000DE4FEF2DF0E0E556FD4F80818883F8014A
:10120000F18081E694E06F2D0E94042AEF2DF0E03A
:10121000888190E0E827F927E556FD4F8081888393
:10122000F801F28081E694E06F2D0E94042AEF2DF0
:10123000F0E0888190E0E827F927E556FD4F8081AE
:101240008883F801F38081E694E06F2D0E94042AE0
:10125000EF2DF0E0888190E0E827F927E556FD4F73
:1012600080818883F801F48081E694E06F2D0E94EC
:10127000042AEF2DF0E0888190E0E827F927E55671
:10128000FD4F80818883F801248135814681578113
:10129000232F342F452F5527F22E81E694E0622F1D
:1012A0000E94042AEF2DF0E0888190E0E827F927DA
:1012B000E556FD4F80818883F80124813581468180
:1012C00057819A0144275527F22E81E694E0622F38
:1012D0000E94042AEF2DF0E0888190E0E827F927AA
:1012E000E556FD4F80818883F80124813581468150
:1012F0005781252F332744275527F22E81E694E086
:10130000622F0E94042AEF2DF0E0888190E0E82708
:10131000F927E556FD4F8081888381E694E060E0FF
:101320000E94042AE881F0E0E556FD4F8081888321
:1013300081E694E060E00E94042AE881F0E0E5564E
:10134000FD4F80818883F801828193810B9718F18A
:101350008AE0A82EB12CA00EB11E750112C0F701B3
:10136000D1907F0181E694E06D2D0E94042AED2D3D
:10137000F0E0888190E0E827F927E556FD4F80816D
:1013800088832E2D2A1930E0F801828193810A97F3
:101390002817390720F3075F1E4F81E694E0F80114
:1013A00060810E94042ADF91CF911F910F91FF90DD
:1013B000EF90DF90BF90AF900895DF93CF93CDB7BC
:1013C000DEB7CA50D1400FB6F894DEBF0FBECDBF16
:1013D0002CE329836A832AE030E03C832B83FC01E1
:1013E00084819581A681B7818D839E83AF83B887E1
:1013F000CE0101960E94E108C65FDE4F0FB6F89459
:10140000DEBF0FBECDBFCF91DF91089585E796E097
:101410006AE773E00E94B32F882331F586E696E6EB
:10142000A6E6B0E48093FD059093FE05A093FF052A
:10143000B093000680E090E0A0E8BFE3809301064F
:1014400090930206A0930306B093040688EE93E0FF
:10145000909306068093050681E8809307068DE841
:10146000809308068DEF25C082E598EBAEE0B0E4EE
:101470008093FD059093FE05A093FF05B0930006B1
:1014800085E89BEEA1E5B0E4809301069093020607
:10149000A0930306B093040680EA94E190930606B5
:1014A000809305068BEF8093070686E680930806F7
:1014B0008AEF809309060895FF920F931F9305E723
:1014C00016E0C8016CE773E00E94B32F80934406D6
:1014D000C8016EE773E00E94B32F80934506C801F0
:1014E00060E873E00E94B32F80932406C8016EE881
:1014F00073E00E94B32F80933C06C8016AE873E052
:101500000E94B32F80933A06C80164E873E00E94FA
:10151000B32F80934606C80166E873E00E94B32F9C
:1015200080934706C8016CE873E00E94B32F809354
:101530002C06C80162E973E00E94B32F809348062D
:10154000C80164E973E00E94B32F80932B06C801A1
:1015500064EF73E00E94B32FF82EC80165EF73E0CB
:101560000E94B32F382F20E02F0D311D30934A06F3
:1015700020934906C80166EF73E00E94B32FF82E4E
:10158000C80167EF73E00E94B32F382F20E02F0DC2
:10159000311D30934C0620934B06C80168EF73E071
:1015A0000E94B32FF82EC80169EF73E00E94B32F99
:1015B000382F20E02F0D311D30934E0620934D061D
:1015C000C8016BEF73E00E94B32F809323061F9135
:1015D0000F91FF900895BC0185E796E00E94B32F1C
:1015E00008956091B0047091B1048091B20490911B
:1015F000B30420E030E040E152E40E94093520E0ED
:1016000030E044EB53E40E943B330E946C350E946F
:10161000A3339B012550304037FF03C09B01215E5F
:101620003F4FACE0B6E0F901E556FC4F80818C936A
:101630002F5F3F4F2432310514F020E030E0119647
:1016400086E0A731B80779F71C9208952F923F9250
:101650004F925F926F927F928F929F92AF92BF92C2
:10166000CF92DF92EF92FF920F931F93DF93CF936E
:1016700000D000D000D0CDB7DEB7182F662E209155
:10168000A6043091A7042A35310530F0C9018D54E4
:101690009F4F89359105E8F437FF02C02D543F4F25
:1016A000C90137FF03C0909581959F4F8A319105FD
:1016B0003CF0F4E48F2E912CE9ED2E2E312C1DC040
:1016C0000A975CF17BE3872E912C62ED262E312C5C
:1016D00020C02B35310514F0235B3040C90137FFA2
:1016E00003C0909581959F4F8A31910554F056E53E
:1016F000852E912C4CED242E312C37E0A32EB12CCD
:1017000015C00A9754F02DE4822E912C94ED292EC9
:10171000312C88E0A82EB12C09C005E0802E912C38
:10172000B8E32B2E312CA9E0AA2EB12C6091A8048D
:101730007091A904882777FD8095982F0E94D63351
:1017400027EA32E94BE25CEB0E9409350E94DD3565
:1017500020E030E040EA50E40E94093520E030E02B
:1017600040E951E40E9409350E946C3520E030E0E8
:1017700044E352E40E946E320E94A333712EFEEBCA
:10178000CF2EFFEFDF2E9B01442737FD4095542FCE
:1017900029833A834B835C83EEE74E2EE4E05E2E92
:1017A0004AEF5FEF240E351E6091A6047091A704E6
:1017B000882777FD8095982F0E94D63325E33AEF4E
:1017C0004EE85CE30E9409350E94DD357B018C0107
:1017D000B601882777FD8095982F0E94D6339B010C
:1017E000AC01C801B7010E9409357B018C016981F8
:1017F0007A818B819C810E94D6339B01AC01C80108
:10180000B7010E946E320E94A3339B01CB01019766
:101810008A35910508F071C062E170E00E9443369C
:101820008B012F5F3F4FAEEEBFEF6A9FC0016B9FF2
:10183000900D7A9F900D1124820F931F62E070E04B
:101840000E9443366D837E83E62CE01A4E2D4C5F5A
:101850008EE794E0672D0E94060500D000D000D0EE
:10186000EDB7FEB73196ADB7BEB712965C924E9209
:10187000119720E031E0338322838D819E81880D92
:10188000991D958384830E9402294DB75EB74A5FF4
:101890005F4F0FB6F8945EBF0FBE4DBF8D819E8126
:1018A0008A159B0554F1043011053CF593E0E90ECF
:1018B000C201672D4E2D0E94060500D000D000D039
:1018C000EDB7FEB73196ADB7BEB712965C924E92A9
:1018D000119720E031E0338322834D815E81420DF8
:1018E000531D558344830E9402298DB79EB70696E7
:1018F0000FB6F8949EBF0FBE8DBFACE0B0E0CA0E2D
:10190000DB1E7394BEE4CB16D10409F04DCF2696AE
:101910000FB6F894DEBF0FBECDBFCF91DF911F9100
:101920000F91FF90EF90DF90CF90BF90AF909F907E
:101930008F907F906F905F904F903F902F90089581
:10194000823010F422E002C0282F220F30E08DB741
:101950009EB708970FB6F8949EBF0FBE8DBFEDB728
:10196000FEB731968EE794E0ADB7BEB712969C9362
:101970008E93119783E091E09383828322573F4FA8
:10198000358324832F5F3F4F378326830E940229AC
:101990008DB79EB708960FB6F8949EBF0FBE8DBF49
:1019A0000895CF93DF93AC01E091B804F091B904AE
:1019B00020910A0630910B06C9018C599F4F8E1752
:1019C0009F071CF4EA01219709C024563040E21712
:1019D000F30714F0EA0102C0EA012196842F90E097
:1019E000C817D90729F085E796E04C2F0E94BA2F37
:1019F000CE01DF91CF9108950F931F9305E716E075
:101A0000C80163EF73E041E00E94BA2FC80164EFA0
:101A100073E043E10E94BA2FC80165EF73E046E02E
:101A20000E94BA2FC80166EF73E040E10E94BA2F0E
:101A3000C80167EF73E047E20E94BA2FC80168EF60
:101A400073E048E80E94BA2FC80169EF73E043E1F0
:101A50000E94BA2F1F910F910895CF92DF92EF92BB
:101A6000FF920F931F937C01D62EC72E0EE714E032
:101A7000C8016E2D4D2D0E946F04C8010E944705BC
:101A800000D000D0EDB7FEB71283018383E391E06D
:101A9000948383830E94F128EDB7FEB712830183FC
:101AA00083E291E0948383830E94F128EDB7FEB72F
:101AB0001283018383E191E0948383830E94F12860
:101AC000EDB7FEB71283018383E091E094838383B3
:101AD0000E94F128EDB7FEB71283018384EF90E0F6
:101AE000948383830E94F1280F900F900F900F90A2
:101AF000C8010E942B05C70101966D2D7C2D0E9407
:101B0000260B1F910F91FF90EF90DF90CF900895DB
:101B1000AF92BF92CF92DF92EF92FF920F931F93FB
:101B2000B82EA62E0E949B3028EE33E040E050E015
:101B30000E94563679018A01AEE7CA2EA4E0DA2E59
:101B4000C6016B2D4A2D0E946F04C6010E944705F5
:101B5000A090D604B090D7048DB79EB744970FB627
:101B6000F8949EBF0FBE8DBFEDB7FEB73196ADB7EF
:101B7000BEB71296DC92CE92119788E091E09383E3
:101B8000828383EB90E095838483C7016CE370E0EC
:101B90000E944336CB016CE370E00E94433697838A
:101BA00086832AE330E031872087C7016CE370E049
:101BB0000E9443369387828785E690E095878487E5
:101BC000C5016CE370E00E942F36CB016CE370E03E
:101BD0000E94433697878687318B208BC5016CE343
:101BE00070E00E942F36938B828B0E9402298DB762
:101BF0009EB744960FB6F8949EBF0FBE8DBFC60128
:101C00000E942B051F910F91FF90EF90DF90CF90D6
:101C1000BF90AF900895EF92FF920F931F93282FDC
:101C2000462FBEE7EB2EB4E0FB2EC701622F0E94C9
:101C30006F04C7010E9447058DB79EB70A970FB67C
:101C4000F8949EBF0FBE8DBF0DB71EB70F5F1F4F1D
:101C5000EDB7FEB7F282E18280E291E0F801938372
:101C600082836091D8047091D9048091DA049091B4
:101C7000DB04209101063091020640910306509149
:101C800004060E940935F80164837583868397836F
:101C900080EB90E0918780870E9402298DB79EB7E4
:101CA0000A960FB6F8949EBF0FBE8DBFC7010E9463
:101CB0002B051F910F91FF90EF9008958F929F92A7
:101CC000AF92BF92CF92DF92EF92FF920F931F934A
:101CD000E82EF62E0EE714E0C8016E2D4F2D0E945F
:101CE0006F04C8010E9447058DB79EB70C970FB6C9
:101CF000F8949EBF0FBE8DBFEDB7FEB73196ADB75E
:101D0000BEB712961C930E93119728E2822E21E003
:101D1000922E938282829DEEA92EB12CB582A4824E
:101D20008091E1049091E204A091E304B091E40475
:101D300086839783A087B18783EFC82ED12CD38663
:101D4000C2860E9402298DB79EB70C960FB6F894F2
:101D50009EBF0FBE8DBFC8010E942B05F394C80122
:101D60006E2D4F2D0E946F04C8010E944705ADB72C
:101D7000BEB71C970FB6F894BEBF0FBEADBFEDB790
:101D8000FEB7319612961C930E931197938282821E
:101D9000B582A4828091E5049091E604A091E704C5
:101DA000B091E80486839783A087B187D386C286E3
:101DB0000E9402298DB79EB70C960FB6F8949EBF6D
:101DC0000FBE8DBFC8010E942B05F394C8016E2D74
:101DD0004F2D0E946F04C8010E944705ADB7BEB7E2
:101DE0001C970FB6F894BEBF0FBEADBFEDB7FEB7E0
:101DF000319612961C930E93119793828282B5822C
:101E0000A4828091E9049091EA04A091EB04B0913E
:101E1000EC0486839783A087B187D386C2860E940D
:101E200002298DB79EB70C960FB6F8949EBF0FBED1
:101E30008DBFC8010E942B051F910F91FF90EF905D
:101E4000DF90CF90BF90AF909F908F9008950F93A9
:101E50001F93282F462F0EE714E0C801622F0E941F
:101E60006F04C8010E9447058DB79EB70A970FB649
:101E7000F8949EBF0FBE8DBFEDB7FEB73196ADB7DC
:101E8000BEB712961C930E93119782E391E0938351
:101E9000828389EB90E0958384838091D404909130
:101EA000D5049783868382E890E0918780870E949B
:101EB00002298DB79EB70A960FB6F8949EBF0FBE43
:101EC0008DBFC8010E942B051F910F910895EF92BD
:101ED000FF920F931F93282F462F3EE7E32E34E007
:101EE000F32EC701622F0E946F04C7010E944705AD
:101EF0008DB79EB70C970FB6F8949EBF0FBE8DBFDF
:101F00000DB71EB70F5F1F4FEDB7FEB7F282E1822C
:101F10008AE391E0F8019383828384EE90E09583D5
:101F200084836091D2047091D304882777FD8095D3
:101F3000982F0E94D6332AE037ED43E25CE30E94FB
:101F40000935F80166837783808791878FE890E071
:101F5000938782870E9402298DB79EB70C960FB691
:101F6000F8949EBF0FBE8DBFC7010E942B051F9125
:101F70000F91FF90EF9008950F931F93282F462FF6
:101F80000EE714E0C801622F0E946F04C8010E948E
:101F900047058DB79EB70C970FB6F8949EBF0FBE3E
:101FA0008DBFEDB7FEB73196ADB7BEB712961C9395
:101FB0000E9311978AE391E09383828382EE90E0FF
:101FC000958384838091CE049091CF04A091D00416
:101FD000B091D10486839783A087B1878EE890E083
:101FE000938782870E9402298DB79EB70C960FB601
:101FF000F8949EBF0FBE8DBFC8010E942B051F9194
:102000000F9108950F931F93282F462F8EE794E08A
:10201000622F0E946F048EE794E00E944705809132
:10202000B504882319F424E431E057C0813019F451
:1020300028E431E052C0823019F42CE431E04DC084
:10204000833019F420E531E048C0843019F424E5E8
:1020500031E043C0853019F428E531E03EC08630D8
:1020600019F42CE531E039C0873019F420E631E06D
:1020700034C0883019F424E631E02FC0893019F4D7
:1020800028E631E02AC08A3019F42CE631E025C078
:102090008B3019F420E731E020C08C3019F424E7AC
:1020A00031E01BC08D3019F428E731E016C08E30C6
:1020B00019F42CE731E011C08F3019F420E831E039
:1020C0000CC0803119F424E831E007C0813119F0E7
:1020D00028E831E002C029E831E08DB79EB70897C3
:1020E0000FB6F8949EBF0FBE8DBFEDB7FEB7319609
:1020F0000EE714E0ADB7BEB712961C930E9311977E
:102100008DE891E09383828380EE90E095838483D1
:10211000378326830E9402298DB79EB708960FB693
:10212000F8949EBF0FBE8DBFC8010E942B051F9162
:102130000F9108950F931F93282F462F0EE714E059
:10214000C801622F0E946F04C8010E9447058DB725
:102150009EB70A970FB6F8949EBF0FBE8DBFEDB71E
:10216000FEB73196ADB7BEB712961C930E9311977A
:1021700082E991E09383828387E890E0958384836A
:102180008091B6049091B7049783868385E290E0AE
:10219000918780870E9402298DB79EB70A960FB655
:1021A000F8949EBF0FBE8DBFC8010E942B051F91E2
:1021B0000F9108950F931F93282F462F0EE714E0D9
:1021C000C801622F0E946F04C8010E9447058DB7A5
:1021D0009EB70A970FB6F8949EBF0FBE8DBFEDB79E
:1021E000FEB73196ADB7BEB712961C930E931197FA
:1021F0008CE991E0938382838091A8049091A90453
:102200009583848380EB90E09783868381EB90E0D5
:10221000918780870E9402298DB79EB70A960FB6D4
:10222000F8949EBF0FBE8DBFC8010E942B051F9161
:102230000F9108950F931F93282F462F0EE714E058
:10224000C801622F0E946F04C8010E9447058DB724
:102250009EB70A970FB6F8949EBF0FBE8DBFEDB71D
:10226000FEB73196ADB7BEB712961C930E93119779
:102270008CE991E0938382838091A6049091A704D6
:102280009583848380EB90E09783868382EB90E054
:10229000918780870E9402298DB79EB70A960FB654
:1022A000F8949EBF0FBE8DBFC8010E942B051F91E1
:1022B0000F9108950F931F93282F462F0EE714E0D8
:1022C000C801622F0E946F04C8010E9447058DB7A4
:1022D0009EB70A970FB6F8949EBF0FBE8DBFEDB79D
:1022E000FEB73196ADB7BEB712961C930E931197F9
:1022F00084EA91E09383828381EE90E095838483E6
:1023000080918502909186029783868385E290E092
:10231000918780870E9402298DB79EB70A960FB6D3
:10232000F8949EBF0FBE8DBFC8010E942B051F9160
:102330000F9108950F931F93282F462F0EE714E057
:10234000C801622F0E946F04C8010E9447058DB723
:102350009EB70C970FB6F8949EBF0FBE8DBFEDB71A
:10236000FEB73196ADB7BEB712961C930E93119778
:102370008CEA91E09383828386EB91E0958384835A
:1023800080ED90E0978386838CE096E0918780874C
:1023900081ED90E0938782870E9402298DB79EB7D6
:1023A0000C960FB6F8949EBF0FBE8DBFC8010E9459
:1023B0002B051F910F9108950F931F93282F462FE0
:1023C0000EE714E0C801622F0E946F04C8010E944A
:1023D00047058DB79EB70A970FB6F8949EBF0FBEFC
:1023E0008DBFEDB7FEB73196ADB7BEB712961C9351
:1023F0000E93119784EC91E0938382838091B004D3
:102400009091B104A091B204B091B30484839583F8
:10241000A683B78380EB90E0918780870E94022992
:102420008DB79EB70A960FB6F8949EBF0FBE8DBFAC
:10243000C8010E942B051F910F9108950F931F93C0
:10244000282F462F0EE714E0C801622F0E946F0468
:10245000C8010E9447058DB79EB70C970FB6F89438
:102460009EBF0FBE8DBFEDB7FEB73196ADB7BEB7FD
:1024700012961C930E9311978CEC91E093838283B8
:1024800086E190E0958384838091CA049091CB0487
:10249000A091CC04B091CD0486839783A087B187A7
:1024A00088E890E0938782870E9402298DB79EB7C3
:1024B0000C960FB6F8949EBF0FBE8DBFC8010E9448
:1024C0002B051F910F910895CF92DF92EF92FF920B
:1024D0000F931F93CF93DF93282F462FCEE7D4E09F
:1024E000CE01622F0E946F04CE010E9447056091C9
:1024F00018067091190680911A0690911B0620917A
:1025000001063091020640910306509104060E9494
:1025100009356B017C0120E030E04AE754E40E9479
:10252000FE341816D4F58DB79EB70C970FB6F894F5
:102530009EBF0FBE8DBF0DB71EB70F5F1F4FADB74C
:10254000BEB71296DC93CE9311978AE391E0F8011F
:10255000938382838EEF90E0958384836091050658
:1025600070910606882777FD8095982F0E94D633B4
:102570009B01AC01C701B6010E943B33D8011696FE
:102580006D937D938D939C931997809109061A966C
:102590008C931A971B961C9221C08DB79EB70C97EF
:1025A0000FB6F8949EBF0FBE8DBFEDB7FEB7319644
:1025B000ADB7BEB71296DC93CE93119786ED91E03E
:1025C000938382838EEF90E095838483C682D78243
:1025D000E086F18680910806828713860E94022990
:1025E000EDB7FEB73C960FB6F894FEBF0FBEEDBF39
:1025F0008EE794E00E942B05DF91CF911F910F9100
:10260000FF90EF90DF90CF900895EF92FF920F939D
:102610001F93282F462F5EE7E52E54E0F52EC701C5
:10262000622F0E946F04C7010E9447058DB79EB7B5
:102630000C970FB6F8949EBF0FBE8DBF0DB71EB797
:102640000F5F1F4FEDB7FEB7F282E1828CEC91E095
:10265000F8019383828389EE90E09583848360916F
:10266000C6047091C7048091C8049091C904209158
:10267000FD053091FE054091FF05509100060E9436
:102680000935F801668377838087918780910706F3
:10269000828713860E9402298DB79EB70C960FB6CB
:1026A000F8949EBF0FBE8DBFC7010E942B051F91DE
:1026B0000F91FF90EF900895EF92FF920F931F9369
:1026C000282F462F6EE7E62E64E0F62EC701622F14
:1026D0000E946F04C7010E9447058DB79EB70C97F3
:1026E0000FB6F8949EBF0FBE8DBF0DB71EB70F5F1C
:1026F0001F4FEDB7FEB7F282E18286ED91E0F8015F
:102700009383828386EE90E0958384836091C204F4
:102710007091C3048091C4049091C5042091010676
:102720003091020640910306509104060E9409353B
:10273000F801668377838087918780910806828776
:1027400013860E9402298DB79EB70C960FB6F89497
:102750009EBF0FBE8DBFC7010E942B051F910F9119
:10276000FF90EF900895EF92FF920F931F93282F01
:10277000462F7EE7E72E74E0F72EC701622F0E94F6
:102780006F04C7010E9447058DB79EB70C970FB61F
:10279000F8949EBF0FBE8DBF0DB71EB70F5F1F4FC2
:1027A000EDB7FEB7F282E18286ED91E0F801938306
:1027B000828387EE90E0958384836091DC0470913E
:1027C000DD04882777FD8095982F0E94D6332091CD
:1027D00001063091020640910306509104060E94C2
:1027E0000935F80166837783808791878091080691
:1027F000828713860E9402298DB79EB70C960FB66A
:10280000F8949EBF0FBE8DBFC7010E942B051F917C
:102810000F91FF90EF9008950F931F93282F462F4D
:102820000EE714E0C801622F0E946F04C8010E94E5
:10283000470580911C060E94A00CC8010E942B0530
:102840001F910F910895EF92FF920F931F93282FDE
:10285000462FEEE7EE2EE4E0FE2EC701622F0E9427
:102860006F04C7010E9447058DB79EB70C970FB63E
:10287000F8949EBF0FBE8DBF0DB71EB70F5F1F4FE1
:10288000EDB7FEB7F282E18286ED91E0F801938325
:1028900082838FE190E09583848360911D0670911F
:1028A0001E0680911F06909120060E94D63320912B
:1028B00001063091020640910306509104060E94E1
:1028C0000935F801668377838087918780910806B0
:1028D000828713860E9402298DB79EB70C960FB689
:1028E000F8949EBF0FBE8DBFC7010E942B051F919C
:1028F0000F91FF90EF9008950F931F93282F462F6D
:102900000EE714E0C801622F0E946F04C8010E9404
:1029100047058DB79EB740970FB6F8949EBF0FBE80
:102920008DBFEDB7FEB73196ADB7BEB712961C930B
:102930000E93119780EE91E09383828383E890E079
:10294000958384838091AC049091AD04A091AE04F2
:10295000B091AF0486839783A087B18784E890E025
:10296000938782878091BC049091BD04A091BE049E
:10297000B091BF0484879587A687B7870E940229F4
:102980008DB79EB740960FB6F8949EBF0FBE8DBF11
:10299000C8010E942B051F910F9108950F931F935B
:1029A000282F462F8EE794E0622F0E946F048EE757
:1029B00094E00E9447058091C104282F30E08230C6
:1029C00030F4F4E0220F331FFA95E1F702C02150F2
:1029D000304000D000D000D0EDB7FEB731960EE702
:1029E00014E0ADB7BEB712961C930E93119780E01A
:1029F00091E093838283358324830E9402298DB7DB
:102A00009EB706960FB6F8949EBF0FBE8DBFC80145
:102A10000E942B051F910F9108950F931F93282F4C
:102A2000462F0EE714E0C801622F0E946F04C80110
:102A30000E9447058DB79EB708970FB6F8949EBFC2
:102A40000FBE8DBFEDB7FEB73196ADB7BEB71296CC
:102A50001C930E93119782EF91E0938382838FE012
:102A600090E0958384838091C004868317820E94BE
:102A700002298DB79EB708960FB6F8949EBF0FBE79
:102A80008DBFC8010E942B051F910F9108950F93D0
:102A90001F930EE714E0C80163E045E00E946F0455
:102AA000C8010E94470500D000D0EDB7FEB71283E1
:102AB00001838DE591E0948383830E94F128EDB733
:102AC000FEB71283018389E491E0948383830E949B
:102AD000F128EDB7FEB71283018383E491E094837C
:102AE00083830E94F1280F900F900F900F90C801E0
:102AF0000E942B051F910F9108950F931F93282F6C
:102B0000462F0EE714E0C801622F0E946F04C8012F
:102B10000E94470500D000D0EDB7FEB712830183B5
:102B200084E791E0948383830E94F1280F900F90B3
:102B30000F900F90C8010E942B051F910F910895CF
:102B4000EF92FF920F931F93CF93DF930E949B30DE
:102B5000209126063091270640912806509129069B
:102B6000261737074807590708F08AC10E949B308B
:102B70006C507E4F8F4F9F4F6093260670932706B1
:102B800080932806909329060EE714E0C8010E945E
:102B90009405C80165E043E00E946F04C8010E94EB
:102BA000470500D000D0EDB7FEB71283018384ED56
:102BB00091E0948383830E94F1280F900F900F90EF
:102BC0000F9080910A0690910B06892B31F080912D
:102BD000210690912206892B81F48091B80490916E
:102BE000B90490930B0680930A068091BA049091E1
:102BF000BB0490932206809321062091BA04309161
:102C0000BB044091210650912206C9018456904090
:102C10004817590724F4809125068F5F08C02C5966
:102C20003F4F241735072CF480912506815080935F
:102C3000250680912506181614F081E003C0843023
:102C40001CF083E08093250680912506823009F4EC
:102C500062C0833009F4BEC0813009F00DC100D0DC
:102C600000D0CEE7D4E0EDB7FEB7D283C1838BECC2
:102C700091E0948383830E94F1288091FC050F905A
:102C80000F900F900F9080FF22C000D000D0EDB7C2
:102C9000FEB7D283C18383EC91E0948383830E9447
:102CA000F12880910A0690910B06845690400F906F
:102CB0000F900F900F902091B8043091B90428170D
:102CC00039070CF0D9C08091FC058E7F21C000D05F
:102CD00000D0EDB7FEB7D283C1838BEB91E0948334
:102CE00083830E94F12880910A0690910B068C59EB
:102CF0009F4F0F900F900F900F902091B80430913C
:102D0000B904821793070CF0B7C08091FC0581606D
:102D10008093FC05B1C000D000D0CEE7D4E0EDB781
:102D2000FEB7D283C18381EB91E0948383830E94B9
:102D3000F1280F900F900F900F9080912306882319
:102D400001F100D000D0EDB7FEB7D283C18387EA8E
:102D500091E0948383830E94F12880910A069091E8
:102D60000B06845690400F900F900F900F9020917B
:102D7000B8043091B904281739071CF510922306BE
:102D800020C000D000D0EDB7FEB7D283C1838AE95E
:102D900091E0948383830E94F12880910A069091A8
:102DA0000B068C599F4F0F900F900F900F90209112
:102DB000B8043091B904821793071CF481E0809322
:102DC000230685E796E06BEF73E0409123060E94AF
:102DD000BA2F52C000D000D0AEE7EA2EA4E0FA2EFF
:102DE000EDB7FEB7F282E18289E891E094838383B4
:102DF0000E94F1288DB79EB708970FB6F8949EBF32
:102E00000FBE8DBF0DB71EB70F5F1F4FEDB7FEB7DB
:102E1000F282E18288EF91E0F801938382836091EE
:102E2000240670E080E090E00E94D43320E030E09F
:102E300040E251E40E943B33F8016483758386834A
:102E4000978386E790E09187808780E290E0938780
:102E500082870E9402298DB79EB70C960FB6F89410
:102E60009EBF0FBE8DBF8091240690E060E873E0A6
:102E70000E94D10C809324068EE794E00E942B05DB
:102E8000DF91CF911F910F91FF90EF9008952F92B6
:102E90003F924F925F926F927F928F929F92AF92EA
:102EA000BF92CF92DF92EF92FF920F931F93DF9327
:102EB000CF93CDB7DEB72A970FB6F894DEBF0FBE1B
:102EC000CDBF8F8368870E949B302091330630915D
:102ED00034064091350650913606261737074807C5
:102EE000590708F051C1809137068823C9F08093B3
:102EF00087021092370680E092E090933906809323
:102F000038060E949B306C507E4F8F4F9F4F6093CE
:102F10003306709334068093350690933606EFC0DF
:102F200080918702282E3324E090B4040091380663
:102F3000109139062091A10429834091C1044E8348
:102F400050912A065D836090CE047090CF048090EB
:102F5000D0049090D1048091240690E040908502A6
:102F60005090860220912B06A22FB0E0BC83AB8349
:102F7000B0912C06BA83F090ED043A8629865C0164
:102F8000CC24B7FCC094DC2CE985FA853196FA870D
:102F9000E98737972CF041E050E05A8749871BC0FA
:102FA00089859A858330910531F1843091053CF40F
:102FB0008130910581F0029709F068C014C0A9859D
:102FC000BA85A530B105C9F1A530B10504F1169750
:102FD00009F05CC043C0B1E0BE1508F457C00DE075
:102FE00012E081E05AC0E981E33009F44FC00AE100
:102FF00012E082E052C0FE81F23008F047C02D811D
:10300000222309F443C007E212E083E046C0C60170
:10301000B5010E94D63320E030E040E251E40E9446
:103020003B339B01AC01C401B3010E9434338823BC
:103030006CF504E312E084E030C04B815C814416FF
:10304000550624F55DE945165FEF5506F9F08A81CE
:103050008823E1F401E412E085E01FC091E09E15B1
:10306000A8F09F1598F4A3E0FA1649F0B4E0FB1617
:1030700049F0E2E0FE1651F40EE412E005C00AE564
:1030800012E002C007E612E086E007C049855A85D3
:103090004215530509F078CF60C0109339060093AC
:1030A00038068093370681E080932D060E949B307E
:1030B00068517C4F8F4F9F4F609333067093340657
:1030C00080933506909336060E949B306056704F71
:1030D0008F4F9F4F60932F06709330068093310679
:1030E0009093320680912E06882321F08EE794E09B
:1030F0000E94940510922E0602C010922D060EE733
:1031000014E0C8016F8148850E946F04C8010E94C5
:10311000470500D000D000D0EDB7FEB73196ADB76F
:10312000BEB712961C930E93119784E792E0938397
:1031300082838091380690913906958384830E941A
:103140000229EDB7FEB736960FB6F894FEBF0FBE54
:10315000EDBFC8010E942B0517C0109339060093DC
:103160003806109237060E949B3020912F0630912E
:10317000300640913106509132062617370748072E
:10318000590708F4BACFBBCF2A960FB6F894DEBF22
:103190000FBECDBFCF91DF911F910F91FF90EF90A8
:1031A000DF90CF90BF90AF909F908F907F906F9067
:1031B0005F904F903F902F900895EF92FF920F9362
:1031C0001F9380913A06843009F056C09091B5045F
:1031D000943008F027C1809143068917A1F190939C
:1031E00043060E949B3060933F0670934006809395
:1031F0004106909342069091430680918802981769
:1032000011F580912E06813091F0813018F08230D6
:10321000B1F413C011E010932E060E949B3061534D
:1032200075478040904030F410933B0608C082E020
:1032300080932E0610923B0602C010922E068EE757
:1032400094E00E9494050E949B3020913F063091AB
:1032500040064091410650914206621B730B840B5D
:10326000950B615D77408040904008F4DBC0809111
:10327000B50480938802D6C0853029F480917D0200
:1032800090917E0214C0863029F480917F02909143
:1032900080020DC0873029F48091810290918202D2
:1032A00006C0883041F4809183029091840290930B
:1032B0003E0680933D0680913C0620913D0630916C
:1032C0003E06882309F04AC0C901895097408F5AA9
:1032D0009440C8F40E949B306153754780409040F1
:1032E00020F481E080933B060CC080913B0688234C
:1032F00041F480912D06882321F48EE794E00E940A
:10330000940582E028C044E0203B340768F48091B3
:103310002E06882349F010923B068EE794E00E9427
:10332000940510922E067EC0205B34402955324011
:1033300008F078C080912E06813009F473C0809126
:103340002D06882309F06EC010923B068EE794E0AC
:103350000E94940581E080932E0664C0215B344076
:1033600008F460C00E949B306153754780409040D4
:1033700008F041C080913B068823E9F5E0903F06C4
:10338000F0904006009141061091420688EE93E0CD
:10339000A0E0B0E0E80EF91E0A1F1B1F0E949B3040
:1033A000E616F70608071907E8F581E080933B0663
:1033B00017C010923B068EE794E00E94940580911E
:1033C0002E06823019F410922E0603C08F5F809370
:1033D0002E0680912E06823018F082E080932E0611
:1033E0000E949B3060933F06709340068093410695
:1033F0009093420617C0E0903F06F090400600917F
:1034000041061091420688EE93E0A0E0B0E0E80E9D
:10341000F91E0A1F1B1F0E949B30E616F7060807BD
:10342000190738F21F910F91FF90EF900895809146
:103430003A06843010F00E94DD1880913B06882304
:1034400019F00E94A01508958091E10380FF08C043
:10345000609147048091450490E070E00E94471716
:1034600080912E06823008F0FDC1A82FB0E0FD014A
:10347000E552FC4F808185FF0BC0FD01E950FC4FF8
:103480006081AB50BC4F8C9190E070E00E940D15B4
:1034900080912E06A82FB0E0FD01E552FC4F8081FF
:1034A00086FF0BC0FD01E550FC4F6081A750BC4F6B
:1034B0008C9190E070E00E94CE1480912A068823BF
:1034C00009F43FC080912E06A82FB0E0FD01E5521F
:1034D000FC4F808187FF0BC0FD01E150FC4F6081F4
:1034E000A350BC4F8C9190E070E00E947C148091BE
:1034F0002E06A82FB0E0FD01E352FC4F808184FF2F
:103500000BC0FD01E95EFB4F6081AB5EBB4F8C9150
:1035100090E070E00E94231480912E06A82FB0E066
:10352000FD01E352FC4F808183FF0BC0FD01ED5E86
:10353000FB4F6081AF5EBB4F8C9190E070E00E94CA
:103540000C1480912E06A82FB0E0FD01E152FC4F33
:10355000808187FF0BC0FD01E15DFB4F6081A35DB2
:10356000BB4F8C9190E070E00E94B31380912E06C7
:10357000A82FB0E0FD01EF51FC4F808183FF0BC00D
:10358000FD01E15BFB4F6081A35BBB4F8C9190E041
:1035900070E00E941E1280912A06882309F46EC0F2
:1035A0008091C104823008F469C080912E06A82F52
:1035B000B0E0FD01ED51FC4F808182FF0BC0FD01A9
:1035C000E55AFB4F6081A75ABB4F8C9190E070E0A9
:1035D0000E94641280912E06A82FB0E0FD01E152F6
:1035E000FC4F808182FF0BC0FD01E55DFB4F6081D8
:1035F000A75DBB4F8C9190E070E00E945C138091BE
:103600002E06A82FB0E0FD01E152FC4F808183FF20
:103610000BC0FD01ED5CFB4F6081AF5CBB4F8C913B
:1036200090E070E00E94051380912E06A82FB0E074
:10363000FD01E352FC4F808181FF0BC0FD01E55F7E
:10364000FB4F6081A75FBB4F8C9190E070E00E94C0
:10365000DC1180912E06A82FB0E0FD01E352FC4F53
:10366000808180FF0BC0FD01E95FFB4F6081AB5F94
:10367000BB4F8C9190E070E00E949A1180912E06D1
:10368000A82FB0E0FD01EF51FC4F808186FF0BC0F9
:10369000FD01E95AFB4F6081AB5ABB4F8C9190E022
:1036A00070E00E945A1180912E06A82FB0E0FD0113
:1036B000E552FC4F808182FF0BC0FD01E151FC4FC0
:1036C0006081A351BC4F8C9190E070E00E941A1170
:1036D00080912E06A82FB0E0FD01E552FC4F8081BD
:1036E00081FF0BC0FD01E551FC4F6081A751BC4F2C
:1036F0008C9190E070E00E94DA1080912E06A82F45
:10370000B0E0FD01E152FC4F808184FF0BC0FD0160
:10371000E55CFB4F6081A75CBB4F8C9190E070E053
:103720000E949A1080912E06A82FB0E0FD01E15270
:10373000FC4F808185FF0BC0FD01E15CFB4F608188
:10374000A35CBB4F8C9190E070E00E9402108091CE
:103750002E06A82FB0E0FD01E552FC4F808183FFCB
:103760000BC0FD01ED50FC4F6081AF50BC4F8C9100
:1037700090E070E00E94BC0F80912E06A82FB0E070
:10378000FD01E152FC4F808180FF0BC0FD01E95D2E
:10379000FB4F6081AB5DBB4F8C9190E070E00E946D
:1037A000670F80912E06A82FB0E0FD01E552FC4F77
:1037B000808184FF0BC0FD01ED5FFB4F6081AF5F37
:1037C000BB4F8C9190E070E00E94270F80912E06F5
:1037D000A82FB0E0FD01ED51FC4F808181FF18C0A2
:1037E00080912306FD01E35AFB4F813049F4A15A31
:1037F000BB4F6C91808190E070E00E940B0E08C07E
:10380000A15ABB4F6C91808190E070E00E945E0EE7
:1038100080912E06A82FB0E0FD01E352FC4F80817D
:1038200087FF0BC0FD01ED5DFB4F6081AF5DBB4FBE
:103830008C9190E070E00E94880D80912E06A82F58
:10384000B0E0FD01E152FC4F808186FF0BC0FD011D
:10385000ED5BFB4F6081AF5BBB4F8C9190E070E004
:103860000E942D0D08958EE794E00E9494050E9419
:1038700047150E94060A0895CF93DF93EC018EE767
:1038800094E00E946B04C817D9073CF08EE794E0DF
:103890000E946004892B09F42397CE01DF91CF9118
:1038A0000895EF92FF920F931F93CF93DF930091B0
:1038B0002E0610E08AEF90E0089F7001099FF00C3F
:1038C000189FF00C1124C7010E94EB0AF801E55281
:1038D000FC4F882319F08081816002C080818E7F37
:1038E000808380912E06C82FD0E0C70102960E94E7
:1038F000EB0ACB51DC4F888380912E06C82FD0E095
:10390000C70104960E94EB0A90E00E943C1CC9513A
:10391000DC4F888300912E0610E0C70188569F4F28
:103920000E94EB0AF801E552FC4F882319F08081D0
:10393000806102C080818F7E808380912E06C82F97
:10394000D0E0C70186569F4F0E94EB0ACF5FDB4F46
:10395000888380912E06C82FD0E0C70184569F4FE0
:103960000E94EB0A90E00E943C1CCD5FDB4F8883F5
:1039700000912E0610E0C70106960E94EB0AF8019E
:10398000E552FC4F882319F08081826002C080815B
:103990008D7F808380912E06C82FD0E0C7010896C6
:1039A0000E94EB0AC751DC4F888380912E06C82FF6
:1039B000D0E0C7010A960E94EB0A90E00E943C1CEE
:1039C000C551DC4F888300912E0610E0C7010C968C
:1039D0000E94EB0AF801E552FC4F882319F0808120
:1039E000846002C080818B7F808380912E06C82FE7
:1039F000D0E0C7010E960E94EB0AC351DC4F8883CA
:103A000080912E06C82FD0E0C70140960E94EB0A95
:103A100090E00E943C1CC151DC4F888300912E062F
:103A200010E0C70142960E94EB0AF801E552FC4FF4
:103A3000882319F08081886002C08081877F80831D
:103A400080912E06C82FD0E0C70144960E94EB0A51
:103A5000CF50DC4F888380912E06C82FD0E0C7015D
:103A600046960E94EB0A90E00E943C1CCD50DC4F31
:103A7000888300912E0610E0C7014E960E94EB0A43
:103A8000F801E552FC4F882319F08081806202C062
:103A900080818F7D808380912E06C82FD0E0C70162
:103AA00080960E94EB0ACB50DC4F888380912E06D3
:103AB000C82FD0E0C70182960E94EB0A90E00E94D6
:103AC0003C1CC950DC4F888300912E0610E0C701D2
:103AD00084960E94EB0AF801E552FC4F882319F006
:103AE0008081806402C080818F7B808380912E06DC
:103AF000C82FD0E0C70186960E94EB0AC750DC4F62
:103B0000888380912E06C82FD0E0C70188960E9436
:103B1000EB0A90E00E943C1CC550DC4F888300916A
:103B20002E0610E0C7018A960E94EB0AF801E552C2
:103B3000FC4F882319F08081806802C080818F77D4
:103B4000808380912E06C82FD0E0C7018C960E94FA
:103B5000EB0AC350DC4F888380912E06C82FD0E03B
:103B6000C7018E960E94EB0A90E00E943C1CC15057
:103B7000DC4F888300912E0610E0C701C0960E949A
:103B8000EB0AF801E352FC4F882319F08081816031
:103B900002C080818E7F808380912E06C82FD0E066
:103BA000C701C2960E94EB0ACB5FDB4F88838091EE
:103BB0002E06C82FD0E0C701C4960E94EB0A90E001
:103BC0000E943C1CC95FDB4F888300912E0610E0E9
:103BD000C701C6960E94EB0AF801E352FC4F882306
:103BE00019F08081826002C080818D7F8083809106
:103BF0002E06C82FD0E0C701C8960E94EB0AC75F07
:103C0000DB4F888380912E06C82FD0E0C701CA966B
:103C10000E94EB0A90E00E943C1CC55FDB4F88834A
:103C200000912E0610E0C701CC960E94EB0AF80125
:103C3000E352FC4F882319F08081846002C08081A8
:103C40008B7F808380912E06C82FD0E0C701CE964F
:103C50000E94EB0AC35FDB4F888380912E06C82F3A
:103C6000D0E0C701805C9F4F0E94EB0A90E00E9469
:103C70003C1CC15FDB4F888300912E0610E0C7011A
:103C8000885B9F4F0E94EB0AF801E352FC4F8823A8
:103C900019F08081806102C080818F7E8083809155
:103CA0002E06C82FD0E0C701865B9F4F0E94EB0A0B
:103CB000CB5EDB4F888380912E06C82FD0E0C701F2
:103CC000845B9F4F0E94EB0A90E00E943C1CC95EFF
:103CD000DB4F888300912E0610E0C7018E5B9F4F5B
:103CE0000E94EB0AF801E352FC4F882319F080810F
:103CF000886002C08081877F808380912E06C82FD4
:103D0000D0E0C7018C5B9F4F0E94EB0ACF5EDB4F78
:103D1000888380912E06C82FD0E0C7018A5B9F4F11
:103D20000E94EB0A90E00E943C1CCD5EDB4F888332
:103D300000912E0610E0C701805B9F4F0E94EB0AA6
:103D4000F801E352FC4F882319F08081806202C0A1
:103D500080818F7D808380912E06C82FD0E0C7019F
:103D60008E5A9F4F0E94EB0AC75EDB4F888380917B
:103D70002E06C82FD0E0C7018C5A9F4F0E94EB0A35
:103D800090E00E943C1CC55EDB4F888300912E06AC
:103D900010E0C7018A5A9F4F0E94EB0AF801E352D4
:103DA000FC4F882319F08081806402C080818F7B62
:103DB000808380912E06C82FD0E0C701885A9F4F7C
:103DC0000E94EB0AC35EDB4F888380912E06C82FCA
:103DD000D0E0C701865A9F4F0E94EB0A90E00E94F4
:103DE0003C1CC15EDB4F888300912E0610E0C701AA
:103DF00082569F4F0E94EB0AF801E352FC4F882342
:103E000019F08081806802C080818F7780838091E3
:103E10002E06C82FD0E0C70180569F4F0E94EB0AA4
:103E2000CF5DDB4F888380912E06C82FD0E0C7017D
:103E30008E559F4F0E94EB0A90E00E943C1CCD5D86
:103E4000DB4F888300912E0610E0C7018E599F4FEB
:103E50000E94EB0AF801E152FC4F882319F080819F
:103E6000816002C080818E7F808380912E06C82F62
:103E7000D0E0C7018C599F4F0E94EB0ACB5DDB4F0E
:103E8000888380912E06C82FD0E0C7018A599F4FA2
:103E90000E94EB0A90E00E943C1CC95DDB4F8883C6
:103EA00000912E0610E0C70182599F4F0E94EB0A35
:103EB000F801E152FC4F882319F08081846002C030
:103EC00080818B7F808380912E06C82FD0E0C70130
:103ED00080599F4F0E94EB0AC75DDB4F888380911A
:103EE0002E06C82FD0E0C7018E589F4F0E94EB0AC4
:103EF00090E00E943C1CC55DDB4F888300912E063C
:103F000010E0C70184579F4F0E94EB0AF801E1526D
:103F1000FC4F882319F08081806802C080818F77F0
:103F2000808380912E06C82FD0E0C70182579F4F13
:103F30000E94EB0AC35DDB4F888380912E06C82F59
:103F4000D0E0C70180579F4F0E94EB0A90E00E948B
:103F50003C1CC15DDB4F888300912E0610E0C70139
:103F60008E569F4F0E94EB0AF801E152FC4F8823C6
:103F700019F08081826002C080818D7F8083809172
:103F80002E06C82FD0E0C7018C569F4F0E94EB0A27
:103F9000CB5CDB4F888380912E06C82FD0E0C70111
:103FA0008A569F4F0E94EB0A90E00E943C1CC95C1D
:103FB000DB4F888300912E0610E0C7018C589F4F7D
:103FC0000E94EB0AF801E152FC4F882319F080812E
:103FD000886002C08081877F808380912E06C82FF1
:103FE000D0E0C7018A589F4F0E94EB0ACF5CDB4F9D
:103FF000888380912E06C82FD0E0C70188589F4F34
:104000000E94EB0A90E00E943C1CCD5CDB4F888351
:1040100000912E0610E0C70186589F4F0E94EB0AC0
:10402000F801E152FC4F882319F08081806102C0C1
:1040300080818F7E808380912E06C82FD0E0C701BB
:1040400084589F4F0E94EB0AC75CDB4F88838091A6
:104050002E06C82FD0E0C70182589F4F0E94EB0A5E
:1040600090E00E943C1CC55CDB4F888300912E06CB
:1040700010E0C70180589F4F0E94EB0AF801E152FF
:10408000FC4F882319F08081806202C080818F7D7F
:10409000808380912E06C82FD0E0C7018E579F4F96
:1040A0000E94EB0AC35CDB4F888380912E06C82FE9
:1040B000D0E0C7018C579F4F0E94EB0A90E00E940E
:1040C0003C1CC15CDB4F888300912E0610E0C701C9
:1040D0008A579F4F0E94EB0AF801E152FC4F882358
:1040E00019F08081806402C080818F7B8083809101
:1040F0002E06C82FD0E0C70188579F4F0E94EB0AB9
:10410000CF5BDB4F888380912E06C82FD0E0C7019C
:1041100086579F4F0E94EB0A90E00E943C1CCD5BAB
:10412000DB4F888300912E0610E0C7018C559F4F0E
:104130000E94EB0AF801EF51FC4F882319F08081AF
:10414000816002C080818E7F808380912E06C82F7F
:10415000D0E0C7018A559F4F0E94EB0ACB5BDB4F33
:10416000888380912E06C82FD0E0C70188559F4FC5
:104170000E94EB0A90E00E943C1CC95BDB4F8883E5
:1041800000912E0610E0C70180559F4F0E94EB0A58
:10419000F801EF51FC4F882319F08081846002C040
:1041A00080818B7F808380912E06C82FD0E0C7014D
:1041B0008E549F4F0E94EB0AC75BDB4F8883809130
:1041C0002E06C82FD0E0C7018C549F4F0E94EB0AE7
:1041D00090E00E943C1CC55BDB4F888300912E065B
:1041E00010E0C7018A549F4F0E94EB0AF801EF517B
:1041F000FC4F882319F08081886002C08081877F0E
:10420000808380912E06C82FD0E0C70188549F4F2D
:104210000E94EB0AC35BDB4F888380912E06C82F78
:10422000D0E0C70186549F4F0E94EB0A90E00E94A5
:104230003C1CC15BDB4F888300912E0610E0C70158
:1042400084549F4F0E94EB0AF801EF51FC4F8823E2
:1042500019F08081806102C080818F7E808380918F
:104260002E06C82FD0E0C70182549F4F0E94EB0A50
:10427000CF5ADB4F888380912E06C82FD0E0C7012C
:1042800080549F4F0E94EB0A90E00E943C1CCD5A44
:10429000DB4F888300912E0610E0C701845A9F4FA0
:1042A0000E94EB0AF801EF51FC4F882319F080813E
:1042B000806402C080818F7B808380912E06C82F0E
:1042C000D0E0C701825A9F4F0E94EB0ACB5ADB4FC6
:1042D000888380912E06C82FD0E0C701805A9F4F57
:1042E0000E94EB0A90E00E943C1CC95ADB4F888375
:1042F00000912E0610E0C70180529F4F0E94EB0AEA
:10430000F801ED51FC4F882319F08081846002C0D0
:1043100080818B7F808380912E06C82FD0E0C701DB
:104320008E519F4F0E94EB0AC75ADB4F88838091C2
:104330002E06C82FD0E0C7018C519F4F0E94EB0A78
:1043400090E00E943C1CC55ADB4F888300912E06EA
:1043500010E0C7018C529F4F0E94EB0AF801ED510B
:10436000FC4F882319F08081826002C080818D7F9C
:10437000808380912E06C82FD0E0C7018A529F4FBC
:104380000E94EB0AC35ADB4F888380912E06C82F08
:10439000D0E0C70188529F4F0E94EB0A90E00E9434
:1043A0003C1CC15ADB4F8883DF91CF911F910F9145
:1043B000FF90EF9008954F925F927F928F929F921D
:1043C000AF92BF92CF92DF92EF92FF920F931F9323
:1043D000DF93CF93CDB7DEB7C854D0400FB6F89473
:1043E000DEBF0FBECDBF0EE714E0C8010E949405EA
:1043F000C80166E049E00E946F04C8010E944705B9
:1044000000D000D0EDB7FEB7128301838FEF91E0AB
:10441000948383830E94F1280F900F900F900F9048
:10442000C8010E942B0500D000D001E614E0EDB7D2
:10443000FEB7128301838FEE91E0948383830E9401
:10444000F12844EE442E41E0542EEE24FF24CC24E7
:10445000DD240F900F900F900F90702E012F39E0F8
:10446000A32EB12CAC0EBD1E4E010894811C911CD4
:1044700081E694E00E94A529982F8D3031F08D308F
:10448000DCF180538230C0F530C01830A1F599813D
:10449000892F8053823078F5913311F490E801C070
:1044A00090E08A81813309F4905C8B81813309F437
:1044B000905E8C81813309F4905F8D81813309F4A2
:1044C000985F8E81813309F49C5F8F81813309F479
:1044D0009E5F8885813309F49F5FF501EE0DFF1D16
:1044E00090830894E11CF11C06C0F401E10FF11D5A
:1044F00090831F5F01C010E0F0E4EF16F104C9F4EF
:104500008EE794E0B601A5010E947F040894C11CC7
:10451000D11C00D000D0EDB7FEB771820283548267
:1045200043820E94F128EE24FF240F900F900F90F9
:104530000F90FFEFCF16D10409F00CF499CFC85BB0
:10454000DF4F0FB6F894DEBF0FBECDBFCF91DF9126
:104550001F910F91FF90EF90DF90CF90BF90AF90A1
:104560009F908F907F905F904F900895DF92EF9291
:10457000FF920F931F93DF93CF93CDB7DEB72A97A8
:104580000FB6F894DEBF0FBECDBF63E0E62EF12C70
:10459000EC0EFD1E53E0D52EADC30E949B30605241
:1045A0007E4480409040C8F40E949B30695873411B
:1045B0008040904090F01A3011F01D3031F480911D
:1045C000F8058F5F8093F80502C01092F80580917E
:1045D000F805833011F40E94DB21812F6EEE74E028
:1045E0000E94F106882311F400E07EC38091F2045A
:1045F0009091F304A091F404B091F5048A3747EC4C
:10460000940749EDA4074BE7B40709F45FC38B3760
:1046100057EC950759EDA5075BE7B50708F0C5C04E
:104620008434EBED9E07E0E7AE07EDE1BE0709F449
:104630004DC38534FBED9F07F0E7AF07FDE1BF07F2
:1046400008F052C0823923EA92072CEEA20724E137
:10465000B20709F4D0C1833933EA93073CEEA307CC
:1046600034E1B307C8F486314AEA940747E3A40764
:104670004BE0B40709F4BFC184305AE9950757ED00
:10468000A5075EE0B50709F4B6C18E5F9B4CA74C49
:10469000B94009F01FC31AC38035FFED9F07FDEE37
:1046A000AF07F8E1BF0709F4E6C281352FED9207A5
:1046B0002DEEA20728E1B20738F488599C42AA419E
:1046C000B64109F007C3A0C18E3C48E4940747E512
:1046D000A4074AE1B40709F4E3C184579B4EAA47F3
:1046E000BB4109F0F7C287C1863AEEE09E07E2E1DE
:1046F000AE07E8E4BE0709F489C2873AFEE09F07E7
:10470000F2E1AF07F8E4BF0740F5823523E29207F4
:1047100026E9A20726E2B20709F43FC2833533E255
:10472000930736E9A30736E2B30738F4825D924C6B
:10473000A248BE4109F0CEC267C1863E55ED95073D
:104740005AEDA50753E3B50709F403C1885F9C4AF6
:10475000AE4EB44309F0BEC2B9C2823EF5E59F0732
:10476000FCE9AF07F6E6BF0709F477C2833E25E50B
:1047700092072CE9A20726E6B20738F48855964B33
:10478000AD4FBA4409F0A6C258C28C3E49E3940723
:1047900046E7A4074BE6B40709F498C280569B4D40
:1047A000AB43BE4609F096C226C18A3BE4E89E07A9
:1047B000E5E2AE07EEEBBE0709F44FC28B3BF4E82F
:1047C0009F07F5E2AF07FEEBBF0708F061C08E3729
:1047D00022E192072AE6A2072BE9B20709F40BC1EE
:1047E0008F3732E193073AE6A3073BE9B30740F579
:1047F00082354AEE940740E8A4074AE8B40709F472
:10480000FAC083355AEE950750E8A5075AE8B50770
:1048100038F4865E964AA642BD4709F05BC240C1A5
:104820008C38F5E89F07F7EAAF07F8E9BF0709F406
:1048300037C18A569E42A246B94909F04BC2E6C129
:1048400080323EE4930739EAA30731EBB30709F45A
:1048500004C281324EE4940749EAA40741EBB4074D
:1048600038F48A57964FA14FBD4909F033C218C199
:104870008A38E7EF9E07E7ECAE07E8EBBE0709F4DE
:10488000C3C0845A9040AB49BA4B09F023C21EC240
:10489000843629ED920720EEA20727EDB20709F42E
:1048A00058C0853639ED930730EEA30737EDB307CF
:1048B00040F5803844E7940740E1A40744ECB4078E
:1048C00009F4A2C0813854E7950750E1A50754ECDC
:1048D000B50738F48C569846A344B24C09F0FAC197
:1048E0004CC18435FDE29F07FFEFAF07F5ECBF0732
:1048F00009F481C086599543A840B24D09F0EAC138
:104900004CC18E343DE593073EE3A30733EEB30776
:1049100009F471C08F344DE594074EE3A40743EECC
:10492000B40738F4865B9342A34AB24E09F0D2C171
:10493000B7C08239E0E79E07E6E8AE07EBEFBE07B7
:1049400009F4C4C1825F9D4EA442BD4F09F0C2C1AB
:104950008DC10E949B306093A2047093A304809346
:10496000A4049093A504D092A1048EEE94E060E19B
:1049700070E00E94C5080E94A3337093A70460935F
:10498000A6048EEE94E064E170E00E94C5080E94E7
:10499000A3337093A9046093A8048EEE94E068E1B9
:1049A00070E00E94C5080E94A3338B017093AB0492
:1049B0006093AA046091AC047091AD048091AE0440
:1049C0009091AF0420E030E040E050E00E943433AA
:1049D000882379F4B801882777FD8095982F0E9465
:1049E000D6336093B0047093B1048093B204909373
:1049F000B30401E070C18091F8048093B404809105
:104A0000F9048093B50466C18EEE94E060E070E036
:104A10000E94C50820E030E048EC52E40E940935CD
:104A20000E94A3337093B7046093B604693C710588
:104A300020F01092B7041092B60480911205909164
:104A400013059093B9048093B80480911405909154
:104A500015059093BB048093BA048091180590913A
:104A6000190590937E0280937D0280911C059091A0
:104A70001D059093800280937F0280911E05909186
:104A80001F0590938202809381028091200590916E
:104A900021059A83898390938402809383021AC1AB
:104AA0006091F8047091F9048091FA049091FB04EC
:104AB0000E94D63320E836E948E15BE40E943B33AC
:104AC0006093AC047093AD048093AE049093AF04F4
:104AD0006091FC047091FD048091FE049091FF04AC
:104AE000D7016C9311967C93119712968C93129721
:104AF00013969C930E94D63320E836E948E15BE4A4
:104B00000E943B336093BC047093BD048093BE0449
:104B10009093BF0480911D058093C00480911C0573
:104B20008093C1048EEE94E060E170E00E94C508BD
:104B30006093B0047093B1048093B2049093B30473
:104B40008EEE94E068E070E00E94C5086093C204B5
:104B50007093C3048093C4049093C5048EEE94E0D4
:104B600064E170E00E94C5086093C6047093C704B6
:104B70008093C8049093C904ADC08EEE94E068E0C1
:104B800070E00E94C50890586093CA047093CB04EB
:104B90008093CC049093CD049DC08EEE94E060E0B1
:104BA00070E00E94C5086093CE047093CF04809398
:104BB000D0049093D1048EEE94E064E070E00E9403
:104BC000C50820E030E048EC52E40E9409350E941C
:104BD000A3337093D3046093D2048EEE94E064E127
:104BE00070E00E94C5080E94A3337093D5046093BF
:104BF000D4048EEE94E068E170E00E94C5080E9443
:104C0000A3337093D7046093D60464C08EEE94E00F
:104C100064E070E00E94C5080E94A333882777FDF6
:104C20008095982F0E94D6336093D8047093D9044E
:104C30008093DA049093DB044DC08EEE94E068E03C
:104C400070E00E94C5080E94A333709561957F4F64
:104C50007093DD046093DC043DC08091580580931F
:104C6000DE04809159058093DF0434C08091F804FC
:104C70008093E0042FC08EEE94E060E070E00E942C
:104C8000C5086093E1047093E2048093E304909379
:104C9000E4048EEE94E064E070E00E94C508609346
:104CA000E5047093E6048093E7049093E8048EEEA5
:104CB00094E068E070E00E94C5086093E904709396
:104CC000EA048093EB049093EC0404C08091040503
:104CD0008093ED0400E08091EF04823229F48EEE9F
:104CE00094E063E20E94DD098EEB90E00E940231C5
:104CF000002331F581E694E00E9475291816190603
:104D0000F4F481E694E00E94A529182F8091A10473
:104D1000882309F062CC41CC1092A10401E0802FDD
:104D200090E02A960FB6F894DEBF0FBECDBFCF91AC
:104D3000DF911F910F91FF90EF90DF90089500E0B9
:104D40002091A2043091A3044091A4045091A504A1
:104D5000205F384D4F4F5F4F2F83388749875A87E1
:104D60000E949B302F81388549855A852617370741
:104D70004807590788F2D3CF1F93CF93DF9385E07D
:104D800090E06CE070E00E947D1568EE73E080E0DA
:104D900090E00E94A93081E694E00E94F229C0E0F0
:104DA000D0E010E0CE016DE171E00E944336892B26
:104DB000A9F41F5E8EE794E0612F4CE00E946F041F
:104DC0008EE794E00E9447058EE794E06EEE0E9425
:104DD00077058EE794E00E942B05105161E070E0AA
:104DE00080E090E00E94A930219687E0C13DD8077D
:104DF000C9F6DF91CF911F91089586E061E00E948E
:104E0000E03108950F931F9386E061E00E94A13185
:104E100001E614E0C80140E051EE60E070E00E945D
:104E2000132910937706009376060E94FD268EE7DD
:104E300094E00E94CD050E94331C64EF71E080E095
:104E400090E00E94A93083EF93E00E94EB0A81304A
:104E500011F00E94FC0C0E945C0A10922E0607C002
:104E60000E94511C80912E068F5F80932E068091A8
:104E70002E068230A8F310922E060E94BC2680E9EE
:104E800094E061ED78E224E630E040E050E000E0BC
:104E90000E94C62F8EE794E00E94940580E994E07A
:104EA0000E942C301F910F9108952F923F924F92A4
:104EB0005F926F927F928F929F92AF92BF92CF92AA
:104EC000DF92EF92FF920F931F93DF93CF9300D067
:104ED00000D0CDB7DEB780912A06882309F4E1C05F
:104EE000E0904F06F0905006009151061091520646
:104EF000C801B7019F7725E33AEF4EE85CE30E94D3
:104F000009350E94383369837A838B839C83C80177
:104F1000B7012091AC043091AD044091AE045091A2
:104F2000AF040E946D321B012C019F7720EC3BE601
:104F300049ED57E40E9409355B016C01609153060D
:104F40007091540680915506909156062091BC04AC
:104F50003091BD044091BE045091BF040E946D3257
:104F60003B014C019F7720EC3BE649ED57E40E9462
:104F7000093529813A814B815C810E9409357B0189
:104F80008C01C601B501A60195010E9409355B019E
:104F90006C01C801B701A80197010E9409359B0166
:104FA000AC01C601B5010E946E320E9490350E948C
:104FB000A33360931D0670931E0680931F06909383
:104FC000200660E070E080E89FE329813A814B8110
:104FD0005C810E943B339B01AC01C201B1010E9484
:104FE000093597FA909497F89094A40193010E9440
:104FF000E13220EE3EE245E652E40E94093520E02F
:1050000030E044EB52E40E946E320E94A3339B01D5
:10501000AC0197FF04C028593E4F4F4F5F4FCA0164
:10502000B901645B70408040904097FF06C0CA01A0
:10503000B9016C547F4F8F4F9F4F0E94D633209100
:10504000B0043091B1044091B2045091B3040E9475
:105050006D320E94A33397FF04C068597E4F8F4F73
:105060009F4F0E94D63320E030E044EB53E40E948F
:105070003B3320E030E040E851E40E9409350E94D3
:105080006C3520E030E040E85FE30E946E320E9421
:10509000A83360931C06613108F46CC010921C06A2
:1050A00069C08091C104823008F464C08091C0045A
:1050B000853008F45FC0A09057068DE18A1508F48A
:1050C00059C0E090C204F090C3040091C404109150
:1050D000C504609158067091590680915A069091C6
:1050E0005B06A80197010E946D329F7720E030E0B7
:1050F00040E05FE30E94FE3418165CF410925706FD
:10510000E0925806F092590600935A0610935B06F7
:1051100031C08A2D8F5F809357068E3159F580916B
:10512000AC049091AD04A091AE04B091AF04809313
:105130004F0690935006A0935106B093520680916B
:10514000BC049091BD04A091BE04B091BF048093B3
:10515000530690935406A0935506B0935606E092DA
:105160005C06F0925D0600935E0610935F0681E098
:1051700080932A060F900F900F900F90CF91DF91A0
:105180001F910F91FF90EF90DF90CF90BF90AF9065
:105190009F908F907F906F905F904F903F902F9057
:1051A00008958091E00480938502109286020E9407
:1051B0004E080E94F10A8EE794E00E9455270E9453
:1051C000171A08950E94B622892B19F00E94D1283F
:1051D000089580E994E00E94143008958FEF9FE7CE
:1051E0000895DF93CF93CDB7DEB7FE0139968D8159
:1051F0009E8161E04F8158859F010E94922BCF9143
:10520000DF910895DF93CF93CDB7DEB7FE013996D6
:105210008D819E8160E04F8158859F010E94922B75
:10522000CF91DF9108950F931F93DC01ED91FC91D5
:105230000288F389E02D20E030E000E010E00995DD
:105240001F910F9108958F92AF92CF92EF92FF929C
:105250000F931F93DF93CF93CDB7DEB7FC0113827B
:10526000128288EE93E0A0E0B0E084839583A68369
:10527000B78383EC93E09183808355874487378796
:105280002687118B008BF38AE28AC48AA58A868AD4
:1052900070E0CB0123E0880F991F2A95E1F79C016C
:1052A0002C59394F308F278B8459994F928F818F8A
:1052B00081E090E002C0880F991F6A95E2F7209183
:1052C0007406282B20937406CF0140E051EE60E075
:1052D00070E00E941329CF91DF911F910F91FF90F1
:1052E000EF90CF90AF908F900895FC01838D88232D
:1052F00019F42FEF3FEF0DC00788F08DE02D2081CE
:10530000318182819381281B390B848195812823E7
:105310003923C9010895FC01838D882319F42FEFE7
:105320003FEF11C0018CF28DE02D2081318182810F
:105330009381281B390B20953095848195812823F2
:1053400039232F5F3F4FC9010895FC01838D8823C6
:1053500061F0A789B08D2D913C91119712968D9196
:105360009C9113972817390721F44FEF5FEFCA017B
:10537000089512968D919C9113971696ED91FC913C
:105380001797E80FF91F408112968D919C91139702
:10539000019614962D913C91159782239323139691
:1053A0009C938E93129750E0E2CFFC01838D88236B
:1053B00051F00788F08DE02D208131818281938129
:1053C0002817390721F42FEF3FEFC9010895828193
:1053D00093810680F781E02DE80FF91F8081282F47
:1053E00030E0F3CFDC015796ED91FC915897828124
:1053F0009381918380835996ED91FC915A97808196
:105400009181938382830895DC015B968C915B97F5
:105410008823A9F15996ED91FC915A972081318109
:105420002F5F3F4F84819581282339235C968C918F
:105430005C97882329F08281938128173907F9F036
:105440008281938128173907D9F380819181068061
:10545000F781E02DE80FF91F60835996ED91FC91DB
:105460005A97318320835296ED91FC915397808116
:1054700056969C91892B808321E030E002C020E089
:1054800030E0C9010895CF93DF93EC011B821A82AB
:105490008A819B81998388831D821C828E819F8152
:1054A000009721F00E94C1031F821E82DF91CF91DD
:1054B00008950F931F938C01DC015296ED91FC919E
:1054C0005397208156968C91569755969C91559757
:1054D000892B80958223808357968D919C91589734
:1054E0000E94432AF801818D928D0E94432AD8019F
:1054F0005B961C921F910F9108950F931F93CF936A
:10550000DF938C01FC01138212828281938191834B
:10551000808341E0A1E0B0E001C04F5FFD01042EB7
:1055200002C0EE0FFF1F0A94E2F79B0182E0613098
:10553000780710F020E032E0E217F30770F3C1E0E3
:10554000D0E002C0CC0FDD1F4A95E2F72197F801A9
:10555000268137812115310541F0848195818C1791
:105560009D0789F0C9010E94C103F801D583C48356
:10557000CE0101960E9417039C01F8019783868350
:1055800080E0232B09F081E0DF91CF911F910F91F3
:105590000895AF92BF92CF92DF92EF92FF920F9356
:1055A0001F93CF93DF937C015A016B01E901DC016A
:1055B0005B968C915B978823F1F02115310539F4C6
:1055C0005796ED91FC915897C481D581219601158C
:1055D000110549F4D7015996ED91FC915A97048130
:1055E00015810F5F1F4FD701ED91FC910088F18964
:1055F000E02DC7010995F7018789908D209711F457
:10560000C0E8D0E0BE010E947D2A882381F0D70146
:1056100059968D919C915A970115110511F400E14D
:1056200010E0B8010E947D2A882309F04DC0D701FF
:10563000ED91FC910088F189E02DC701099567C0C3
:10564000D7015096ED91FC915197B0E0AB16B1EEB9
:10565000BB06B0E0CB06B0E0DB0609F454C081E045
:1056600090E0D70154960C9002C0880F991F0A94BD
:10567000E2F7808360E079E08DE390E0A601950198
:105680000E9478362150304040405040CA01B90154
:1056900022E030E040E050E00E947836D7011C96CE
:1056A000ED91FC911D9730831E96ED91FC911F9713
:1056B0002083D7015296ED91FC91539780815596A6
:1056C0009C91892B808323C0D7015996ED91FC9141
:1056D0005A97138212828281938191838083579695
:1056E000ED91FC915897138212828281938191836C
:1056F000808381E05B968C931A141B041C041D04A8
:105700000CF49ECFD6CF108220E130E0C7CFDF91DE
:10571000CF911F910F91FF90EF90DF90CF90BF90AE
:10572000AF9008952F923F924F925F926F927F9227
:105730008F929F92AF92BF92CF92DF92EF92FF92A1
:105740000F931F93DF93CF93CDB7DEB764970FB658
:10575000F894DEBF0FBECDBF3C01688B5A8B498BDE
:1057600069011C01AE014F5F5F4F5C8B4B8BE98978
:10577000FA89488940FD659140FF6191FA8BE98B78
:10578000662309F4D7C3653249F440FD859140FF93
:105790008191FA8BE98B8532B1F40CC06A3051F4F7
:1057A000D301ED91FC910190F081E02DC1016DE0FC
:1057B00009956AE0D301ED91FC910190F081E02D13
:1057C000C1010995D4CF982F10E088249924103274
:1057D000B0F49B3269F09C3228F4903251F093324D
:1057E00071F40BC09D3239F0903349F4116028C038
:1057F0001260146025C0186023C0106121C017FD1D
:105800002BC0892F80538A3078F416FF06C0BAE087
:105810009B9E902C1124980E13C0EAE08E9E802C43
:105820001124880E10620CC09E3221F416FD82C332
:10583000106406C09C3611F4106802C0983661F4FA
:10584000E989FA89488940FD959140FF9191FA8B49
:10585000E98B992309F0BBCF892F8554833020F43D
:10586000812F8061905E07C0892F8556833008F0B4
:10587000E6C1812F8F7E86FD02C076E0972E6FE312
:10588000F62EF822953619F450E4F52A07C096361C
:1058900019F480E8F82A02C091109A94F7FE0BC020
:1058A0009BE3991520F427E05CE3B52E0DC0B92CDD
:1058B000B39427E009C0A7E0A91520F447E0942E8F
:1058C00027E001C0292DBB24F6013496FD87EC8723
:1058D000D6016D917D918D919C91AE014F5F5F4F8F
:1058E0000B2D0E943F026C010981E02FF0E0FF8741
:1058F000EE8700FF05C0FE85F3FD02C01DE209C072
:10590000F1FE02C01BE205C0F2FC02C010E001C0C3
:1059100010E28E859F858C709070892B09F444C0AD
:10592000112311F483E001C084E0881510F088246D
:105930000EC0881AF3FC0BC0D301ED91FC910190CD
:10594000F081E02DC10160E209958A94A9F7112345
:1059500049F0D301ED91FC910190F081E02DC1015E
:10596000612F0995BE85B3FF03C008E013E012C0A4
:105970000CE013E00FC0E114F10409F06052D30110
:10598000ED91FC910190F081E02DC10109950F5F2F
:105990001F4F05C0EF2CFF24B0E1EB22FF24F801DC
:1059A0006491662341F748C1F7FE13C0BC0CFE8525
:1059B000F4FF04C08A81813309F4BA941B141CF0EB
:1059C000BB24B3942DC048E04B1550F538E0B32EFE
:1059D00027C0F6FC25C0892D90E08C159D054CF064
:1059E0005CEFC5165FEFD50624F080E8F82A01C009
:1059F0009A94992049F0E2E0F0E0EC0FFD1FE90DE8
:105A0000F11D80818033A1F3F7FE0AC0B92CB39455
:105A1000892D90E0C816D90614F0992401C09C186D
:105A2000F7FC03C025E030E009C01C141D041CF085
:105A300021E030E003C096012F5F3F4F112311F0AA
:105A40002F5F3F4F992029F0892D90E00196280F74
:105A5000391F882D90E02817390714F0882401C0D9
:105A6000821A4F2C5524C20189709070892B59F0ED
:105A70000CC0D301ED91FC910190F081E02DC101AA
:105A800060E209958A948820A1F7112349F0D30197
:105A9000ED91FC910190F081E02DC101612F0995FC
:105AA00043FE0BC00CC0D301ED91FC910190F0813D
:105AB000E02DC10160E309958A948820A1F7F7FEE3
:105AC00051C08601D7FE02C000E010E076010894C4
:105AD000E11CF11CE01AF10AE1E0F0E0EC0FFD1F1F
:105AE000EE0EFF1E26014B185108892D90E0AA24C6
:105AF000BB24A81AB90AFFEF0F3F1F0749F4D301CF
:105B0000ED91FC910190F081E02DC1016EE20995CB
:105B1000C016D10634F0401651061CF4F70160811E
:105B200001C060E3015010400894E11CF11C0A150B
:105B30001B054CF0D301ED91FC910190F081E02D1B
:105B4000C1010995D8CF0C151D0541F48A81863312
:105B500020F4853319F4BE85B4FF61E3D301ED91E0
:105B6000FC9165C06A81613309F00F7ED301ED912C
:105B7000FC910190F081E02DC10109959920E1F09F
:105B8000D301ED91FC910190F081E02DC1016EE215
:105B9000099512E0E1E0F0E0EC0FFD1FE10FF11DCF
:105BA00060811F5FD301ED91FC910190F081E02DA8
:105BB000C10109959A9471F7D301ED91FC9101907F
:105BC000F081E02D44FC02C065E601C065E4C1013E
:105BD0000995D7FC05C0C114D10441F404FF06C0E7
:105BE000D094C194D108D3946DE201C06BE2D3018B
:105BF000ED91FC910190F081E02DC101099560E3E8
:105C000005C06F5FE6EFFFEFCE0EDF1EFAE0CF16A6
:105C1000D104BCF7D301ED91FC910190F081E02D0E
:105C2000C1010995D301ED91FC916C2D605D01904E
:105C3000F081E02DC1010995CC84DD8478C19336D3
:105C400031F0933799F0933509F061C023C0F60124
:105C5000808189835E010894A11CB11C42E050E060
:105C6000C40ED51E21E0E22EF12C12C0D601AD905B
:105C7000BC9016FD03C06FEF7FEF02C0692D70E08E
:105C8000E2E0F0E0CE0EDF1EC5010E9424047C019C
:105C90001F7713C0D601AD90BC9016FD03C06FEF07
:105CA0007FEF02C0692D70E0E2E0F0E0CE0EDF1E73
:105CB000C5010E9419047C01106813FF0BC023C0AA
:105CC000D301ED91FC910190F081E02DC10160E2E2
:105CD00009958A94882D90E0E816F90688F313C098
:105CE000F50117FD659117FF61915F01D301ED91FA
:105CF000FC910190F081E02DC101099581108A94F9
:105D00000894E108F108E114F10451F710C1943648
:105D100011F0993699F517FF0AC0F60120813181FB
:105D20004281538184E090E0C80ED91E0CC0D60198
:105D30008D919C919C01442737FD4095542FE2E0C2
:105D4000F0E0CE0EDF1E9FE6F92EF12257FF09C0CC
:105D500050954095309521953F4F4F4F5F4FF0E85C
:105D6000FF2ACA01B901AE014F5F5F4F2AE030E060
:105D70000E94E101E82E4B89E41A41C0953721F4D5
:105D80001F7E2AE030E01CC0197F9F3661F09037FB
:105D900020F4983509F0CEC00FC0903739F098370D
:105DA00009F0C8C004C028E030E00AC0106114FD4A
:105DB000146020E130E004C014FD166020E132E000
:105DC00017FF08C0D6016D917D918D919C91E4E003
:105DD000F0E008C0D6018D919C91BC0180E090E07C
:105DE000E2E0F0E0CE0EDF1EAE014F5F5F4F0E949B
:105DF000E101E82EFB89EF1A8FE7F82EF122F6FE7B
:105E00000BC04EEFF422E91438F4F4FE07C0F2FCA4
:105E100005C05FEEF52202C01E2D01C0192DF4FE53
:105E20000DC0FE01EE0DF11D8081803319F489EE65
:105E3000F82208C01F5FF2FE05C003C08F2D8678D0
:105E400009F01F5F0F2DF3FC18C0F0FE13C01815EA
:105E500010F09E2C0FC09E2C980C911A182D0AC081
:105E6000D301ED91FC910190F081E02DC10160E240
:105E700009951F5F1815A0F304C0181510F4811AB6
:105E800001C0882404FF17C0D301ED91FC9101905B
:105E9000F081E02DC10160E3099502FF29C0D30123
:105EA000ED91FC910190F081E02D01FD02C068E7C9
:105EB00012C068E510C0802F8678D1F001FF02C0C3
:105EC0006BE201C060E2F7FC6DE2D301ED91FC9161
:105ED0000190F081E02DC10109950AC0D301ED9137
:105EE000FC910190F081E02DC10160E309959A9445
:105EF000E914A0F3EA94D301ED91FC91A1E0B0E0A4
:105F0000AC0FBD1FAE0DB11D0190F081E02DC101A0
:105F10006C910995EE2071F70AC0D301ED91FC91C7
:105F20000190F081E02DC10160E209958A948820FA
:105F3000A1F71DCC64960FB6F894DEBF0FBECDBF9F
:105F4000CF91DF911F910F91FF90EF90DF90CF9055
:105F5000BF90AF909F908F907F906F905F904F9089
:105F60003F902F900895F999FECF72BD61BDF89AC8
:105F700080B50895F999FECF1FBA72BD61BD40BDCD
:105F80000FB6F894FA9AF99A0FBE08950F93FC0190
:105F90006115710511F480E011C0218332834383C0
:105FA0005483728761870170000F000F000F80819A
:105FB000877F802B82608B7F808381E00F910895A3
:105FC000CF93DF93EC010E949B309B01AC018D814C
:105FD0009E81AF81B885281739074A075B0728F4E7
:105FE000888184FD02C060E00DC089819A81AB8107
:105FF000BC81820F931FA41FB51F8D839E83AF8327
:10600000B88761E0222757FD23953327442755277A
:10601000922F91709295907F88818F7E892B8883B3
:10602000862FDF91CF910895CF93DF93EC01888184
:1060300082FF0FC0CE010E94E02F882351F0E98536
:10604000FA85309709F00995888183FF02C08B7F1C
:106050008883DF91CF910895CF93DF93EC018985F9
:106060009A85892BE1F089819A81AB81BC81009767
:10607000A105B105A1F00E949B3029813A814B8195
:106080005C81260F371F481F591F2D833E834F8386
:106090005887888184608F7E888381E001C080E09A
:1060A000DF91CF9108951F920F920FB60F92112496
:1060B0002F933F938F939F93AF93BF9380917C06D1
:1060C00090917D06A0917E06B0917F06309180066A
:1060D0000196A11DB11D232F2D5F2D3720F02D57C7
:1060E0000196A11DB11D2093800680937C0690939C
:1060F0007D06A0937E06B0937F06809178069091EE
:106100007906A0917A06B0917B060196A11DB11D7A
:106110008093780690937906A0937A06B0937B06D5
:10612000BF91AF919F918F913F912F910F900FBE93
:106130000F901F9018958FB7F89420917C0630919E
:106140007D0640917E0650917F068FBFB901CA013E
:1061500008959B01AC017FB7F894809178069091E7
:106160007906A0917A06B0917B0666B5A89B05C01A
:106170006F3F19F00196A11DB11D7FBFBA2FA92F46
:10618000982F8827860F911DA11DB11D62E0880FF1
:10619000991FAA1FBB1F6A95D1F7BC012DC0FFB77D
:1061A000F8948091780690917906A0917A06B09142
:1061B0007B06E6B5A89B05C0EF3F19F00196A11D2F
:1061C000B11DFFBFBA2FA92F982F88278E0F911DC1
:1061D000A11DB11DE2E0880F991FAA1FBB1FEA9500
:1061E000D1F7861B970B885E9340C8F22150304050
:1061F0004040504068517C4F211531054105510503
:1062000071F60895019739F0880F991F880F991F2B
:1062100002970197F1F70895789484B5826084BD60
:1062200084B5816084BD85B5826085BD85B581609A
:1062300085BDEEE6F0E0808181608083E1E8F0E0FA
:106240001082808182608083808181608083E0E829
:10625000F0E0808181608083E1EBF0E08081846008
:106260008083E0EBF0E0808181608083EAE7F0E00A
:10627000808184608083808182608083808181606E
:1062800080838081806880831092C10008951F926E
:106290000F920FB60F9211242F933F934F935F935A
:1062A0006F937F938F939F93AF93BF93EF93FF93DE
:1062B0008091810690918206892B29F0E0918106D8
:1062C000F09182060995FF91EF91BF91AF919F9157
:1062D0008F917F916F915F914F913F912F910F908F
:1062E0000FBE0F901F9018951F920F920FB60F922E
:1062F00011242F933F934F935F936F937F938F93CB
:106300009F93AF93BF93EF93FF93809183069091F8
:106310008406892B29F0E0918306F0918406099583
:10632000FF91EF91BF91AF919F918F917F916F916D
:106330005F914F913F912F910F900FBE0F901F9043
:106340001895CF93DF93482F50E0CA018E5B9C4F86
:10635000FC013491425D5C4FFA018491882369F11C
:1063600090E0880F991FFC01E05FFC4FA591B4916C
:10637000FC01E65EFC4FC591D491662351F42FB722
:10638000F8948C91932F909589238C9388818923FD
:106390000BC0623061F42FB7F8948C91932F9095D5
:1063A00089238C938881832B88832FBF06C09FB756
:1063B000F8948C91832B8C939FBFDF91CF9108959C
:1063C000482F50E0CA018A5A9C4FFC012491CA010F
:1063D0008E5B9C4FFC019491425D5C4FFA013491BD
:1063E000332309F440C0222351F1233071F02430CB
:1063F00028F42130A1F0223011F514C02630B1F07C
:106400002730C1F02430D9F404C0809180008F7708
:1064100003C0809180008F7D8093800010C084B580
:106420008F7702C084B58F7D84BD09C08091B00094
:106430008F7703C08091B0008F7D8093B000E32FF1
:10644000F0E0EE0FFF1FE65EFC4FA591B4912FB771
:10645000F894662321F48C919095892302C08C9145
:10646000892B8C932FBF0895CF92DF92EF92FF92EA
:106470000F931F93CF93DF937C016B018A01C0E0E0
:10648000D0E00FC0D6016D916D01D701ED91FC9167
:106490000190F081E02DC7010995C80FD91F015067
:1064A00010400115110571F7CE01DF91CF911F91B9
:1064B0000F91FF90EF90DF90CF900895CF93DF93EF
:1064C0000E940C310E940227C0E0D0E00E94E22826
:1064D0002097E1F30E940000F9CF5058BB27AA276C
:1064E0000ED041C201D230F006D220F031F49F3FED
:1064F00011F41EF4C0C10EF4E095E7FBB6C1E92F1C
:1065000054D280F3BA17620773078407950718F00F
:1065100071F49EF56CC20EF4E0950B2EBA2FA02DEF
:106520000B01B90190010C01CA01A0011124FF2740
:10653000591B99F0593F50F4503E68F11A16F0403B
:10654000A22F232F342F4427585FF3CF469537953A
:106550002795A795F0405395C9F77EF41F16BA0BFF
:10656000620B730B840BBAF09150A1F0FF0FBB1FAD
:10657000661F771F881FC2F70EC0BA0F621F731FF6
:10658000841F48F4879577956795B795F7959E3F53
:1065900008F0B3CF9395880F08F09927EE0F9795E1
:1065A00087950895A1D158F080E891E009F49EEF15
:1065B000A2D128F040E851E059F45EEF09C05BC178
:1065C00016C2E92FE078F1D168F3092E052AC1F34C
:1065D000261737074807590738F00E2E07F8E02529
:1065E00069F0E025E0640AC0EF6307F8009407FA59
:1065F000DB01B9019D01DC01CA01AD01EF934AD075
:10660000B2D10AD05F91552331F02BED3FE049E440
:1066100050FD49EC63CF0895DF93DD27B92FBF7795
:1066200040E85FE31616170648075B0710F4D92FFA
:10663000E9D19F938F937F936F93BCD2E8E6F0E00C
:106640001DD191D12F913F914F915F91EED1DD23DB
:1066500049F09058A2EA2AED3FE049EC5FE3D07898
:106660005D274DDFDF917FC1DCD008F481E0089524
:106670004AD1E39589C10CD076C13DD140F034D1E7
:1066800030F021F45F3F19F0F0C05111B1C1F3C0F7
:106690008CD198F39923C9F35523B1F3951B550B6E
:1066A000BB27AA2762177307840738F09F5F5F4FE5
:1066B000220F331F441FAA1FA9F333D00E2E3AF026
:1066C000E0E830D091505040E695001CCAF729D040
:1066D000FE2F27D0660F771F881FBB1F261737078F
:1066E0004807AB07B0E809F0BB0B802DBF01FF27BF
:1066F00093585F4F2AF09E3F510568F0B6C078C1AD
:106700005F3FECF3983EDCF3869577956795B795F8
:10671000F7959F5FC9F7880F911D9695879597F913
:106720000895E1E0660F771F881FBB1F621773078C
:106730008407BA0720F0621B730B840BBA0BEE1FA1
:1067400088F7E095089504D06894B11151C1089577
:1067500034D188F09F5790F0B92F9927B751A0F006
:10676000D1F0660F771F881F991F1AF0BA95C9F7E5
:1067700012C0B13081F03BD1B1E0089538C1672F2C
:10678000782F8827B85F39F0B93FCCF38695779595
:106790006795B395D9F73EF490958095709561957E
:1067A0007F4F8F4F9F4F0895E89409C097FB3EF4A9
:1067B00090958095709561957F4F8F4F9F4F99234E
:1067C000A9F0F92F96E9BB279395F69587957795CC
:1067D0006795B795F111F8CFFAF4BB0F11F460FF8C
:1067E0001BC06F5F7F4F8F4F9F4F16C0882311F0E4
:1067F00096E911C0772321F09EE8872F762F05C0F8
:10680000662371F096E8862F70E060E02AF09A9592
:10681000660F771F881FDAF7880F9695879597F987
:106820000895990F0008550FAA0BE0E8FEEF161621
:106830001706E807F907C0F012161306E407F50774
:1068400098F0621B730B840B950B39F40A2661F0E8
:10685000232B242B252B21F408950A2609F4A1408B
:10686000A6958FEF811D811D089597F99F6780E898
:1068700070E060E008959FEF80EC0895DF93CF9380
:106880001F930F93FF92EF92DF927B018C0168942C
:1068900005C0DA2EEF01C9D0FE01E894A59125913B
:1068A000359145915591AEF3EF0129DEFE01970137
:1068B000A801DA9479F7DF90EF90FF900F911F9184
:1068C000CF91DF9108959F938F937F936F93FF9361
:1068D000EF939B01AC019DD0EF91FF91CFDF2F9102
:1068E0003F914F915F9195C000240A9416161706A8
:1068F00018060906089500240A94121613061406B1
:1069000005060895B8CF59D0E8F3E894EFEFBB2718
:106910003FE048EC5FE76B3D73078407950708F19C
:10692000FF279F57B25A6A4D7F40894CF04032F49E
:10693000BE556542704F8643FF4F0894EE1F91503D
:1069400030F0BB0F661F771F881FFF1FEBCF9EE73E
:10695000882332F0BB0F661F771F881F9A95C1F7F7
:106960009395E09565C1092E0394000C11F48823DA
:1069700052F0BB0F40F4BF2B11F460FF04C06F5FF7
:106980007F4F8F4F9F4F0895EF93E0FF06C0A2EA1D
:106990002AED3FE049EC5FEBB2DDE5DF0F900394B9
:1069A00001FC9058E5E9F0E08ECF57FD9058440F78
:1069B000551F59F05F3F71F04795880F97FB991F5E
:1069C00061F09F3F79F0879508951216130614061B
:1069D000551FF2CF4695F1DF08C0161617061806A8
:1069E000991FF1CF86957105610508940895E89483
:1069F000BB2766277727CB0197F9089512DF08F4A4
:106A00008FEF08959B01AC0160E070E080E89FE3A8
:106A100032CE0BD0A8CF68DF28F06DDF18F09523B9
:106A200009F023CF28CF1124E3CFBFDFA0F3959F38
:106A3000D1F3950F50E0551F629FF001729FBB2765
:106A4000F00DB11D639FAA27F00DB11DAA1F649F11
:106A50006627B00DA11D661F829F2227B00DA11DC4
:106A6000621F739FB00DA11D621F839FA00D611D4A
:106A7000221F749F3327A00D611D231F849F600D6B
:106A8000211D822F762F6A2F11249F5750408AF0A4
:106A9000E1F088234AF0EE0FFF1FBB1F661F771F30
:106AA000881F91505040A9F79E3F510570F0DDCEF0
:106AB0009FCF5F3FECF3983EDCF386957795679523
:106AC000B795F795E7959F5FC1F7FE2B880F911D4E
:106AD0009695879597F9089570DFE0F09E37D8F086
:106AE0009639B8F49E3848F4672F782F8827985F36
:106AF000F9CF86957795679593959539D0F3B62F0D
:106B0000B1706B0F711D811D20F487957795679586
:106B1000939573C08DC06CCF11F40EF4ACCE88C0C9
:106B20004CDFD0F39923D9F3CEF39F57550B87FF52
:106B30008FD056959795B0E020F4660F771F881F89
:106B4000BB1F1F930F9300249001A0018001F0014F
:106B5000A0E80E0F1F1F0A1E511D601B710B80093C
:106B6000B50B48F4600F711F801DB51F0E1B1F0B66
:106B70000A0A510907C02E0F3F1F4A1F0E0F1F1F81
:106B80000A1E511D660F771F881FBB1FA695F7951C
:106B9000E795F8F60617170708065B07211D311D54
:106BA000411D0F911F91B901842F9158880F96951F
:106BB000879508959B01AC012CCFDF93D92FA3DEDD
:106BC000E695D7952AED3FE049E45FE3B33A6207E3
:106BD000730784079507D7952AF0A2EA49EC9068D5
:106BE0008EDCC1DEE3EBF0E06EDEDD0F0BF00ADFE2
:106BF000DD0F0BF49058DF910895882371F477230B
:106C000021F09850872B762F07C0662311F499271F
:106C10000DC09051862B70E060E02AF09A95660FC7
:106C2000771F881FDAF7880F9695879597F908954B
:106C30009F3F49F0915028F4869577956795B795D1
:106C40009F5F80389F4F880F9695879597F9089595
:106C500091505040660F771F881FD2F70895AA1BE6
:106C6000BB1B51E107C0AA1FBB1FA617B70710F037
:106C7000A61BB70B881F991F5A95A9F78095909569
:106C8000BC01CD01089597FB092E07260AD077FD98
:106C900004D0E5DF06D000201AF4709561957F4F8F
:106CA0000895F6F7909581959F4F0895A1E21A2EC9
:106CB000AA1BBB1BFD010DC0AA1FBB1FEE1FFF1FA0
:106CC000A217B307E407F50720F0A21BB30BE40BF0
:106CD000F50B661F771F881F991F1A9469F7609537
:106CE0007095809590959B01AC01BD01CF010895F1
:106CF00097FB092E05260ED057FD04D0D7DF0AD00A
:106D0000001C38F450954095309521953F4F4F4FDA
:106D10005F4F0895F6F790958095709561957F4F38
:106D20008F4F9F4F0895EE0FFF1F0590F491E02DB8
:066D30000994F894FFCF66
:106D360025630025632563002563253269256325C0
:106D46003032697C25632532692563253032690036
:106D560025352E3066256300256325312E356625BB
:106D660063002563253569256300256325352E32A5
:106D7600662563006D616E007374310073743200B2
:106D8600737433007374340073743500737436008F
:106D960070682000636C200076722000686C20000A
:106DA60061702000727462006C616E007070200069
:106DB600706F6900616320000061742000256325FF
:106DC6007300256325332E30692563002534692534
:106DD60063256300256325336925630025737C25B8
:106DE60063257325630020C0C0C0C0C0C7C0C0C033
:106DF600C0C0200025342E30662563002563253368
:106E06002E3066256300256325352E306625630002
:106E160025632531312E36667C25632531312E36A4
:106E2600660025632532690025332E316625630009
:106E36002020202020202020202020200020206428
:106E4600697361726D6564202000206E6F20746521
:106E56006C20636F6D2000206E6F20677073206654
:106E660069782000202062617474206C6F7720207E
:106E7600006C696E6B207175616C697479006D6167
:106E860067207761726E696E67006D616720637255
:106E960069746963616C00206D6167202065727298
:106EA6006F722000257300200089060000E803E8C1
:106EB60003E803E8039DFF01640000000077053442
:106EC60032750478047B047E04EE2800070E091C44
:106ED6001B1215383F363124232A2D70777E796CA4
:106EE6006B6265484F464154535A5DE0E7EEE9FC54
:106EF600FBF2F5D8DFD6D1C4C3CACD90979E998C44
:106F06008B8285A8AFA6A1B4B3BABDC7C0C9CEDB74
:106F1600DCD5D2FFF8F1F6E3E4EDEAB7B0B9BEABE3
:106F2600ACA5A28F88818693949D9A2720292E3B13
:106F36003C35321F18111603040D0A5750595E4B83
:106F46004C45426F68616673747D7A898E87809539
:106F5600929B9CB1B6BFB8ADAAA3A4F9FEF7F0E523
:106F6600E2EBECC1C6CFC8DDDAD3D4696E676075D3
:106F7600727B7C51565F584D4A4344191E171005C3
:106F8600020B0C21262F283D3A33344E49404752F6
:106F9600555C5B7671787F6A6D64633E3930372263
:106FA600252C2B0601080F1A1D1413AEA9A0A7B293
:106FB600B5BCBB9691989F8A8D8483DED9D0D7C203
:106FC600C5CCCBE6E1E8EFFAFDF4F3C2C0C0C1C020
:106FD600C0C1C0C0C4C0C0C1C0C0C1C0C0C3C0C0A1
:106FE600C1C0C0C1C0C0C5C0C0C1C0C0C1C0C00052
:106FF600000000042A34327529A529D529F2298BE7
:08700600291329592AC92A00A7
:00000001FF
